:020000041100E9
:10300000002373B52B4D2C4C28006361022601F080
:103010006BF94021FE2221742800284B009601F014
:10302000B5F9002836D1217CFF222800244B0096D8
:1030300001F0ACF900282DD1224BA2899A4226D169
:10304000E389214A93420DD1204B6361204B2268D2
:10305000002A03D1002B01D043CB43C4280001F048
:1030600081F973BD1B4A934201D00023EFE71A4B4D
:103070001A4A1B68934206D9C02304222800217CE7
:103080009B0001F0F9F9114B6361154BDFE7002359
:103090002374EAE7CC233821AC2228009B01217459
:1030A00001F0EAF90028F2D10E4B63610E4BE38187
:1030B0000E4BCCE7643CFF1F0C5CFF1F185CFF1F2E
:1030C0001A5CFF1F595900008305000015410011CB
:1030D00008BD001182150000305CFF1F871300003F
:1030E00014BD0011CD410011AAAAFFFFFCBC0011C4
:1030F000F7B5164B0192C318021D002000938823D8
:103100005B05D3181B685C1C1AD09CB2402C18D8E5
:103110008D781E0CAC466746CD782D023D43AE42FD
:1031200006D1019800280ED110000C70240A4C70B2
:1031300003249BB20733A343D218009B9A42DED3E9
:10314000FEBD4432F9E71000FAE7C046FC0F00006C
:10315000802213B503000324019189B25201073183
:103160009B18A14304305A1A88235B05C3181B68B7
:10317000591C03D190429241104016BD99B240298A
:1031800007D80B000733A343C0189042ECD30020AC
:10319000F3E74430F9E7134B134A1B68126810B584
:1031A000FA24934201D81A00F824104BE4021B6859
:1031B0009A4210D813000E4A12689A420ED3013375
:1031C00007D1F823DB029C4203D10A49054808F0E5
:1031D0000FFD200010BDFC24E402ECE7FE24E40215
:1031E000F7E7C04600C0071100D0071100E0071143
:1031F00000F00711FFFFFF7FF0B59BB015000490B2
:103200000391402A00D9A0E006AB59801A80FFF74D
:10321000C2FF0400042816D9002206A9FFF768FFA0
:10322000052810D906AB1B88AB420CD1002D07D066
:10323000514B2A000499C01808F0DAFB002802D18B
:1032400001201BB0F0BD06AB1D8020000699FFF7E2
:103250007FFF041E7BD1069B0793FFF79CFF802313
:103260005B01C618802307001B039E4201D3F8268A
:10327000F60288235B05F31801931B68013302D023
:10328000019808F0BDFA3D49019808F0B1FC3B1DDA
:103290000293331D05938822029B52059B181B68DD
:1032A00008935A1C3CD044219AB20091402A04D879
:1032B0000320D11D814389B2009103991B0C8B42DD
:1032C00024D0402A22D80122300008A9FFF710FF9D
:1032D000021E1BD1380008A9FFF70AFF04000428CA
:1032E00031D9009A059B9B1880225201B218934253
:1032F00040D288235B05C118009A09A808F0D8FBC2
:103300001D4B009A09A9F01808F052FC009A029B84
:103310009446634402931A4B029AFB189A42BAD31A
:1033200088235B05FC1821680198013908F060FCCE
:10333000200008F065FA039A07AB5A80300007991D
:10334000FFF706FF0400002C03D1002079E70428D2
:10335000FBD988235B05E018069908F049FC032394
:10336000EA1C9A4300D16BE7034B0499E01808F07C
:103370001FFC65E70424ECE704000011FFFFFF7F5A
:10338000F80F0000F7B505001400402A21D80027E7
:1033900001AE71803780FFF7FEFE042816D93A008F
:1033A0003100FFF7A5FE042810D93688BC420BD0A7
:1033B000BD4209D0221CB44200D9321C064B92B245
:1033C000C118280008F074FB30B2FEBDC04300B243
:1033D000FBE703204042F8E70400001137B5042260
:1033E00004000D0001A81649FFF7CCFF02000428D5
:1033F0000BD1019BA34208D3AB4204D0104901A8D2
:103400000195FFF7F9FE01203EBD0E4C2368200018
:10341000019308F0F5F9019920000139019108F0B4
:10342000E7FB80235B01E418074B9C42EED10422AA
:10343000034901A80195FFF7DFFE0020E4E7C0463D
:103440005555000000C007110000081130B589B0C3
:1034500008F00EFA10226946254808F049F9254B74
:10346000009A9A420ED1019B029A0F2B33D8002169
:1034700001240698013B08D2002900D00292029B49
:10348000013331D10023029325E0551CF2D1020013
:103490002100EFE710341022200004A908F028F9D9
:1034A000029B013301D1069B0293882304995B059B
:1034B000C918059B06981A03120B049105928142C4
:1034C00003D02B4201D108F0F3FA019B013B019399
:1034D000019B002BDED1029B002B03D004930498A8
:1034E0004168084709B030BDE025014C2D03EFE7E6
:1034F00000000111504859368022F8B5964C974B80
:10350000D200002120001C6008F092F92300944AA8
:1035100088331A60934B1A786A23002A00D011333B
:10352000E3620A232365904B37221B780821A363AB
:103530008E4B6018E361102323628D4B3B25636142
:10354000C823DB00A36123008C331A602823013ACF
:10355000E26321646364C267043A201DC2672000ED
:10356000BC3005602000C03001602000C430036022
:1035700020000635CC3005602000083DC8300560CD
:103580002000D03002602200D43211602200D832F4
:10359000136022000226E032200016604222DC3056
:1035A000026020001B3DE43005602000E83001602F
:1035B0002000EC30036023000520F4331860230062
:1035C000F0331A602300183290331A6023009433CA
:1035D000196023001E3A98331A60AF23DB00236082
:1035E000644BFA252363644B6448A3642300B93217
:1035F000FC33FF32AD00A260E56022611D60A06275
:103600007320E0656D386065A065FA2796203F015C
:103610008000E76465625960A0660920E0660020CA
:10362000616757496666E167564E57492667A06746
:103630000F601527676027001A219C373960270023
:103640000731A037396027004B49A837396021007E
:10365000F8310D6021006427A4310F6021005F3F25
:10366000AC310F602100033FB0310F602700B43749
:103670003D00C8272F6027003825B83738609D6087
:10368000424D96215D64424D8900DD61414D1962D4
:103690005D62F53DFF3D9D621E253949DD66596637
:1036A000996499673C49DE651E6618675867D96753
:1036B000BE233A495B00E1508130394BFF30235043
:1036C00004302150C42149006350C623E4205B002C
:1036D000E2500433E2503349334A344BD160344929
:1036E000800019503349E938FF3819503249043005
:1036F000195032493248D16132491163324951631C
:103700001900F4310860CE20304940001160304982
:10371000195019002F48F83108602F49D1658221CE
:103720002E4A89005A501A002D490832D1671A00D2
:103730002C49B432116088212B4A89005A501A0052
:103740002A49883211602A4ADA6408F0C9F801204F
:1037500007F07EFFF8BDC0460004FF1FB05EFF1FEC
:103760009069FF1FA03EFF1F4A0AFF1F3A07000093
:1037700080C3C9019A02000050C300006A1800000B
:1037800088130000204E0000F009FF1F6509FF1F8D
:1037900068100000C4090000DC05000040420F0072
:1037A00010270000D91AFF1FFC00FF1F0000FF1F99
:1037B0008127FF1FC52AFF1F5D29FF1F251EFF1F31
:1037C0007523FF1F411EFF1FED1FFF1FB11DFF1FB0
:1037D0000124FF1FE924FF1FD918FF1FB923FF1F72
:1037E000C921FF1FD521FF1FB11CFF1F691DFF1F2E
:1037F0009D1CFF1FF0B5022501245D4B91B01D708B
:1038000002935C4B5C4E1C705C4F03933368002149
:103810002800FB7006F008FE280006F0FFFC0023DD
:10382000984205D0FA78552A02D0332A00D093E086
:10383000336007F0DDFFFFF75FFE1F220124002148
:103840004F4B10AD1A704F4B1C704F4B19704F4BB4
:1038500019689143163A0A431A6060221968914325
:10386000403A0A431A6007F0CBFE07F001FFC1207F
:10387000FF21474B80001A588A431A50C5229200F4
:1038800098588843BF390143995098584149084096
:103890008021C9010143802099509958C00509022F
:1038A000090A0143995080213B48490108F068F812
:1038B00003232200394901940093394808F0E0F8C5
:1038C0002C22384905A808F0F3F805AC6178207877
:1038D000023406F0C3FCA542F8D1334C334B2268C6
:1038E00003201A40A023DB021343236080232268B5
:1038F0009B041343236022682D4B1A4080239B03B3
:10390000134323602B4A2C4B934200D8012007F02D
:1039100007FF08F075F880232268DB041343236057
:10392000029B187808F0FCF8039B1878C0B208F0E6
:103930001FF808F0CDF82149042008F009F806F036
:10394000A7FE00F0ABF800F0EDFD00F095FE00F0F2
:103950000FFA002011B0F0BD00932100174A042097
:1039600007F0B6FF8023DB059C62FFF76FFD60E781
:103970004A0AFF1FA03EFF1F34F000403C5CFF1FBF
:10398000480AFF1F490AFF1F680AFF1FBCF00040DA
:1039900000E100E0FF00FFFFA43EFF1F2851FF1FD2
:1039A000A44EFF1F20BC001114F00040FF7FF8FF61
:1039B000FFFF9FFF0080FF1F9069FF1F3B00010872
:1039C00070B500252549264A26484D6308CA1B05BF
:1039D0001B0DED188242F9D100268022224B920560
:1039E0008B630921214B224C1E62224B1120DA6786
:1039F000214BDA688A43DA609A6820490A409A6063
:103A0000266008F0EDF8112007F00AFF636C1C4AED
:103A1000134063641B4C1C4A6C43200C0400642359
:103A200090420AD8FA223300D200904205D9174BAF
:103A30000A21C01807F09CFEC3B2154A1120137268
:103A4000D48007F0FDFE134B1B78002B04D1124BE2
:103A50001021187807F0DCFF70BDC046000005405B
:103A60008807054000080540FF01000000F0004005
:103A70000038004004E100E03CF00040FFDFFFFFC1
:103A8000FFFDFFFFAE060000B70B000030F8FFFFA0
:103A9000245CFF1F5E5EFF1F5C5CFF1F002210B5F1
:103AA0001100112007F094FE10BD0000F8B50023AE
:103AB0000925374F374C3B62E3681120AB43E36085
:103AC00007F0AEFE112008F08BF8112007F0B8FDCA
:103AD0004023226880261343236080236268DB0230
:103AE00013436360A3682C4A3343A360A368280090
:103AF0001340A3608023A2689B0113431022A3609C
:103B0000236C022193432364236C0F3A13432364F1
:103B100080235B013B62226B204B1A402263626B65
:103B20001A406263A26B1A40A263E26B1340E36324
:103B3000E3681B4A1340E36006F090FB2800012174
:103B400006F0A0FC8023174A9B00516C11200B4308
:103B5000536407F0F5FDFD21134B144A89005A50B8
:103B60008023C720E26B5B031343E363E3688000B9
:103B70001D430F4BE56019580E4A11408022120276
:103B80000A431A50802292051A600B4B5E63F8BDFF
:103B900000F000403CF00040FFFFDFFFEFFFEFFFD1
:103BA000FFFF7FFF003800400000FF1FC1390011F8
:103BB00000E100E0FF00FFFF0000054030B503A872
:103BC00004880B20002C0ED14968074D08784978ED
:103BD000090201430A20A94205D1012120001980D0
:103BE000024B1B7A137030BD192A0000245CFF1FA2
:103BF000F7B5150008AA16884A680F4F147852784E
:103C0000120222430A24BA4214D10122DBB20192E9
:103C100000962A0007F076FC041E0BD1074B1B68A8
:103C2000002B07D068782A780002104342425041A6
:103C3000013098472000FEBD02290000A85BFF1F4D
:103C400030B5012503790400BFB02B4211D00A49D9
:103C5000408806F0C3FF28420BD0084B01A95B8DBA
:103C60004D800B80064B00221B7A60880B7104F09C
:103C7000BDF83FB030BDC046A05BFF1FD83AFF1F64
:103C8000245CFF1F10B50549054806F05DFF0421BF
:103C9000044A054806F01AFF10BDC046A05BFF1F8E
:103CA000FFFF00004CBC0011D83AFF1F10B50248BE
:103CB00004F01EFF10BDC046413C0011062310B5A4
:103CC000837010330371443B43712A33837144334F
:103CD000C37100230222012103720E4B0270417056
:103CE0001C8881724472197A0273C1729A78427385
:103CF000DA7882730322C2731A7902745A79427491
:103D00000C2282749A79C274DB7903751123C37013
:103D1000152010BD245CFF1F10B5142007F000FE15
:103D2000124B14220021186007F082FD002007F0DA
:103D3000E7FD012007F0DCFD022007F0B1FD0320C4
:103D400004F07AF9042006F08FF9052003F0B8FB9F
:103D5000062004F085F8072001F04EFA082006F04E
:103D600095FE092001F036F810BDC046AC5BFF1F80
:103D700007F016FE012007F013FD07F079FE0000A2
:103D8000094B10B50400984205D0012904D1200048
:103D9000064906F0D9FE10BD0229FCD1013904F014
:103DA00065FE0028F3D0F6E7FEFF0000D25BFF1FA0
:103DB00070B50D7A100004AA2C0016881022144049
:103DC000154220D1002E20D10A78022A18D14A6843
:103DD000517815780E4A09022943914205D00D4ABF
:103DE000914209D01C800A2404E014220A491A8056
:103DF00007F05EFE200070BD0C2208491A80F7E72C
:103E00001C800124F6E70824F4E70B24F2E7C046FF
:103E1000F3FF0000F4FF0000303DFF1F2CBD001138
:103E200010B504000749084806F08EFE074804F064
:103E30009FFD0020E40704D50721054A054806F048
:103E400045FE10BDD25BFF1FFFFF0000813D00114A
:103E500090BC00111C3BFF1F00B50C4BBFB01A7883
:103E60000B4902A800F0C2FC6B4680B2D880002843
:103E700009D06A46074B01A91B889380064B002294
:103E8000188803F0B3FF3FB000BDC046B05BFF1F12
:103E9000B15BFF1F763BFF1F803CFF1F00B50C4B43
:103EA000BFB01A780B4902A801F0E6FE6B4680B25B
:103EB000D880002809D06A46074B01A95B8D938002
:103EC000064B0022188803F091FF3FB000BDC046AA
:103ED000DA5BFF1FDB5BFF1F1C3BFF1F803CFF1FEC
:103EE000F7B50E00377A1C0008AB11003D001A88A8
:103EF00020231D401F423CD13378022B3BD17368F5
:103F00001F785B781B023B431E4FBB4208D01E4FFD
:103F1000BB4214D01D4DAB4221D00A252800FEBD66
:103F2000002A2AD1142C2AD82200F06807F0C0FDFC
:103F3000174B1C70012CF1D9FFF7B0FFEEE7002AF8
:103F40001BD1202C1BD82200F06807F0B1FD114BCB
:103F500004211C70104B187807F05AFDDEE7E3B21D
:103F60000124009201940A00310007F0CBFA050009
:103F7000D4E70825D2E70125D0E70B25CEE70D25AC
:103F8000CCE7C046F3FF0000F4FF00000229000068
:103F9000DA5BFF1FB05BFF1F5C5CFF1F332310B5B4
:103FA000040003700A220749013007F081FD064B27
:103FB0000F201B681A0AE37222731A0C1B0E62731D
:103FC000A37310BD245CFF1F4C5CFF1F30B501259F
:103FD00003790400BFB02B4213D00B49408806F090
:103FE000FDFD28420DD06A46084B02A81B8893802D
:103FF000FFF7D4FF6B46D8800022608801A903F048
:10400000F5FE3FB030BDC046D25BFF1F763BFF1FC1
:1040100010B5024804F06CFD10BDC046CD3F001144
:1040200070B5160004AA148805AA15784A68507855
:10403000117800022A4A0843801805284BD807F057
:10404000CFFC03131E29343F0720042C0BD8052274
:10405000121BAA4200D92A0022491A8030000919ED
:1040600007F026FD002070BD0720112CFBD812227E
:10407000121BAA4200D92A001B491A80EEE707202A
:104080000E2CF0D80F22121BAA4200D92A00174981
:104090001A80E3E70720032CE5D80422121BAA426A
:1040A00000D92A0012491A80D8E70720032CDAD851
:1040B0000422121BAA4200D92A000E491A80CDE719
:1040C0000720032CCFD80422121BAA4200D92A00B1
:1040D00009491A80C2E700220A201A80C3E7C046B5
:1040E000DCD5FFFFDBBC0011F85BFF1FCBBC001170
:1040F000C6BC0011C1BC0011BCBC001110B50D2123
:10410000024A034806F0E2FC10BDC046B0BC0011F4
:104110008C3BFF1FF0B50024274E85B03000B471F2
:1041200000F0E2F8254D264BEA89297C9A422FD1EE
:104130000423300003AA00F057F90400300000F017
:1041400011F90123B371002C34D16B4699892B6886
:10415000C9BA4B4329891B4A1B145B1853806B4611
:10416000D9896B6849BA89B24B4369891B0C5B18C2
:104170001548191C1BB2834200DD011C0B0400D53D
:1041800000211388918001331380200005B0F0BD19
:104190000227220003AB3000009700F0F7F80E234F
:1041A0000400297C0122300000976B4400F0EEF8F7
:1041B0000443C3E71C00E8E7643CFF1F0C5CFF1FDF
:1041C00083050000245CFF1F0F27000073B5234EFA
:1041D000300000F089F8224D07236A463000297C20
:1041E00000F002F904003000002C33D16B461B783C
:1041F0007F2B2FD800F0B6F86B46D878F023020456
:104200001B031A406B469B8816495BBA9BB21A4344
:104210002B68000953432A891B0C9B184B806B4663
:104220005A789B7812031B011A436B68024353436D
:104230006A891B0C9B180C481A1C1BB2834200DDB8
:10424000021C130400D500220B888A8001330B80E6
:10425000200076BD00F086F80124F9E7643CFF1FDA
:104260000C5CFF1F245CFF1F0F27000070B5114C72
:10427000237C002B0FD0382B0ED10F4D280000F0DF
:1042800033F8CC23AC222800217C9B0100F0F4F809
:10429000280000F067F870BD084BE2899A42FAD115
:1042A000054D280000F020F800222800217C00F0B5
:1042B000C5F8EDE70C5CFF1F643CFF1F83050000A1
:1042C00010B5084B1A7C002A09D05B69002B06D078
:1042D0009847041E01D0FEF793FE200010BD012474
:1042E000F9E7C0460C5CFF1F70B5C17905000C00F2
:1042F000631E9C411A4BE402E41849000460C9B2F1
:10430000007906F0F5F8E979687949000131C9B218
:1043100006F0EEF8E8790930C0B207F091F9002311
:10432000E36661332360AA795B3B002A0ED02268E2
:104330009A43023B134323600A23E361073323625A
:1043400000232363A3630133E36370BD22689A43B0
:10435000022313432360462363610633A361EFE71F
:104360000050004070B5002504000368DD66C07988
:104370000930C0B207F054FA2900207906F054F849
:104380002900607906F050F870BD0000F8B51E00F5
:1043900006AB1D78002304681700E366616007F030
:1043A00067FA01238022E3662B0027615200013B5C
:1043B00008D207F095FB08200A4A1168002D03D1A6
:1043C0002800F8BD2261F2E7236F034203D023697E
:1043D000013D3370013613685B1A032BEED90125BA
:1043E000EEE7C0466008FF1F70B51C00002305689B
:1043F0001600EB66696007F03BFA01238022EB664A
:1044000023005200013B08D207F06AFB08200A4A49
:104410001168002C03D1200070BD2A61F2E72B6FD8
:10442000034203D02B69013C3370013613685B1AD9
:10443000032BEED90124EEE76008FF1F002370B5BF
:1044400004681500E366616007F012FA0123E36671
:10445000256107F045FB8020064A80001168636BE8
:10446000034205D113685B1A032BF8D9012070BDF4
:104470000020FCE76008FF1F70B51D0000230468E2
:104480001600E366616007F0F3F90123E366266135
:104490000F33626B1A42FCD02B0A23611023626B2C
:1044A0001A42FCD0EDB2256107F01AFB8020074AC2
:1044B00080001168636B034205D113685B1A032BFC
:1044C000F8D9012070BD0020FCE7C0466008FF1F3E
:1044D00070B51E00002305681400EB66696007F0E4
:1044E000C7F90123A619EB660F33B4420ED107F0CA
:1044F000F7FA80200A4A800011686B6B03420CD1E6
:1045000013685B1A032BF8D9012070BD217829614B
:10451000696B1942FCD00134E7E70020F5E7C0469B
:104520006008FF1F10B5084CE368002B08D18022FB
:10453000064B52021B689B186360054B1B68236087
:1045400007F0F6FAA06010BD4C5CFF1FC8F00040F9
:10455000CCF0004070B5184A936A916A9942FBD139
:1045600016498A689A421FD39A1A8B60144B012607
:10457000186893B2D202D20E4343424300204C68E3
:104580001B0A1B1912029B180E4C0A684B60551C23
:10459000A3420CD8002801D04B600A600A4A13607D
:1045A00008680A4B186070BD581E821ADDE7084A79
:1045B00030009B182A00EAE700F000404C5CFF1F27
:1045C000140AFF1F40420F00C8F00040CCF000402A
:1045D000C0BDF0FF70B51F4C23793F2B01D93F239D
:1045E00023711D4B22791A701878C0B207F0C8FAEF
:1045F00018231A491A4A0B801A4913800B805380DA
:10460000A379194980200B800C21938001334B43FF
:10461000164D191C0001834200D9011C2980D1804C
:104620006379002B11D101336371237A012B01D8F7
:10463000022323726279237A0D4853430A21584397
:1046400007F096F80B4D286070BDA02BEDD9A02384
:10465000EAE7C046405CFF1F480AFF1F7E3CFF1F81
:104660004C3EFF1F7C3CFF1F7A3CFF1F783CFF1F26
:1046700071020000305CFF1FF8B514210020FEF726
:10468000ADFE114C011E114D09D10C22104BC1CBB6
:10469000C1C4280007F0CCF8FFF79CFFF8BD0C223E
:1046A00020000C49FEF76EFE0C2802D0084B43CBCD
:1046B00043C40C2228000849FEF764FE0C28EBD006
:1046C0000C220021E5E7C046405CFF1F0C5CFF1F89
:1046D00020BD0011FC0C0000F50C0000F0B51D4CD5
:1046E0008022A5440400882069465201400507F055
:1046F00067FA902212016A441300200032C832C3C4
:1047000016C816C38023144C144FA6689B0333436A
:10471000A3603B6007F0D4F88823A0685B05C0184D
:1047200007F06EF80025882329008022A0685B0529
:10473000C01840196944520007F03AFA8023013545
:10474000FF355B019D42EED1A6603E60044B9D4467
:10475000F0BDC046FCEFFFFFC03DFF1F9808FF1FE4
:1047600004100000F0B5040087B0002825D068468A
:1047700007F006F81B4C022806D1062269462000E5
:1047800007F036F9002816D06946002301250F26C8
:104790002F00E25C013310091030874038002F00F1
:1047A000324097403A0002434A610439062BEFD168
:1047B0006846FFF793FF07B0F0BD182269460A4824
:1047C00007F0FEF96A46A300D358013305D018223A
:1047D000FF21684607F02CF8EAE70134062CF1D1F6
:1047E000E9E7C0466509FF1F00090011F0B5002583
:1047F00004000E0085B0AA4200D186E04B1C087868
:1048000001934B788978377909021943F3783F0689
:104810001B040B431F43039720706570252800D1AC
:1048200096E033D8112813D807F062F969002801FF
:10483000280128012801AA00B800B1002801280198
:10484000280128012801280128012801020122014C
:10485000232800D1DBE0DB2800D031E1042A00D896
:10486000ACE01025052A05D0551F2A003800711D1F
:1048700007F01EF905223100200007F019F92A007F
:104880003900601D07F014F905353EE0562859D06F
:1048900010D8332800D19DE0552839D02628DAD108
:1048A0009D4B2900132218001D0006F0C1FFFEF7E2
:1048B000A7FB5CE0712800D177E0722800D180E08E
:1048C000602800D18BE0DC28C5D1022A00D875E031
:1048D0007378BFB26370B378A370032A05D0033A2C
:1048E000390092B2F01CFEF787FC10223900E01C60
:1048F000FEF748FDC51C002807DA60705CE00C225A
:104900002000864907F0D4F80C25280005B0F0BD3A
:10491000013A834D0C2A13D8002A0AD028000199A5
:1049200007F0C6F8FFF756FE0C2228007D49FEF777
:1049300063FC29000C22601C07F0BAF80D25E4E79F
:104940000C22EBE7764D784B2A0043CB43C2E9E7D4
:10495000013A714D0C2A11D8002A08D0019928007B
:1049600007F0A6F80C2228007049FEF745FC290044
:104970001322601C07F09CF81425C6E70C22EDE713
:1049800005226B49601C07F093F80625BDE712224B
:104990006849601C07F08CF81325B6E708226649C1
:1049A000601C07F085F80925AFE77178F02905D874
:1049B000624B188801F0BCFD0225A6E7FF23637057
:1049C000FAE75F4B012A03D072789A706270F3E7BE
:1049D0009B78F4E72000FFF7E1FA050095E7013A3C
:1049E000574B584D082A0DD8002A0DD00121280018
:1049F0005970019907F05CF801F072F8082229005B
:104A0000601CCEE70822F1E700225A70F6E7042A7C
:104A100004D94D4D2F6007F08BF8A860FFF79AFD81
:104A20000422039003A9601C07F042F805256CE7F7
:104A3000464D062A15D906222800019906F0D8FF0E
:104A400000280ED006220199280007F031F806222E
:104A50003F492800FEF7D0FB0123394A91780B43E8
:104A6000937029000622601C07F022F807254CE706
:104A7000012AA3D07078FFF775FE9DE7012800D0CA
:104A8000E9E6931E334F1A2B04D87378002B09D113
:104A900000F014F9304B39001D78601C6A1E07F0D5
:104AA00007F832E7551E2A000199380007F000F890
:104AB0002A49AAB23800FEF79FFB00F035F9E9E772
:104AC000DA281DD1042A00D878E7082A15D9B37945
:104AD00072791B021343F27912041A43337A1B06CC
:104AE00013433B603B68052231002000039306F02E
:104AF000DFFF0422601D03A953E7FE236370F1E783
:104B0000DE2800D05AE7511E012A01D10025FCE61B
:104B1000019800F0CBFFF9E70C5CFF1F2CBD0011E2
:104B2000405CFF1FFC0C000020BD0011F50C0000D4
:104B3000185CFF1FF85BFF1FC43DFF1F803CFF1F79
:104B40003C5CFF1F1D3DFF1F4C5CFF1F6509FF1FE5
:104B5000ADAC00003D5EFF1F3B5EFF1FAEDE000000
:104B600070477047020010B5094B0A32094C92B2E7
:104B7000DA815A8298811882207802F03FFB042261
:104B8000054B012120781A7006F042FF10BDC04687
:104B90004E3DFF1F865EFF1F855EFF1F013870B50B
:104BA000042809D806F01CFF030928081200234B2B
:104BB0000221187806F02CFF70BD204B08211878D0
:104BC00006F09EFF00221E4B1A72F5E78022002499
:104BD0001B4B1A4D52001A8108211A682878DC7282
:104BE00006F0EEFD2100287806F0BAFF012000F063
:104BF00063FE00F075FFDFE7104B0821187806F020
:104C00007FFF1048FFF75AF80F4B104A9B7900209E
:104C100093800F4A13808022094B5200D8721A8168
:104C200000F04AFE00F05CFF0A4B9B78002BC3D0DB
:104C3000094A136006F0B4FFBEE7C0465C5CFF1F84
:104C4000305CFF1F893CFF1F405CFF1F4C3EFF1F75
:104C50007A3CFF1F3C5CFF1F34F0004010B5012977
:104C60000BD1022809D1054B1B78002B05D0262239
:104C7000034B04485A72FFF775FF10BD5E5EFF1FBD
:104C8000305CFF1FC40900000300F0B50A4D8E1808
:104C9000B14202D152008018F0BD0C782F6824096F
:104CA0003C5D0F271C700C7801313C402F683C5D47
:104CB0005C700233ECE7C046743CFF1F0E22114BC0
:104CC00010B51A700D23104C10492370093A043B9B
:104CD0000F48637006F0ECFE2D2301220D490E48AB
:104CE000E371FFF7D1FF01220C49FFF7CDFF01224D
:104CF0000B49FFF7C9FF00220A491000FEF77CFAB2
:104D000010BDC0465A5EFF1F3B5EFF1FDBBC00119B
:104D10003D5EFF1F6709FF1F435EFF1F6609FF1F00
:104D20006509FF1FAEDE000070B5124C1322200093
:104D30001149FEF727FB114D002817DDAB78002B3A
:104D400014D0431C2B7009236B70002300190370CF
:104D5000287829000130C0B206F03AFF29782200F5
:104D60000139C9B2002005F0CFFD70BDFFF7A6FFE5
:104D7000EEE7C0463D5EFF1FAEDE00003B5EFF1F5C
:104D800010B5114B1A781870002A0ED000280BD1DC
:104D90000E4B1A78062A07D85423D340DB0703D5D5
:104DA0000B4B187802F02AFA10BD0028FCD0074BF4
:104DB0001B78012B02D0033B022BF5D8044B0121B9
:104DC000187806F025FEEFE75E5EFF1F855EFF1F89
:104DD000865EFF1F70B54A4E4A4A4B49307002202A
:104DE00005F034FC00F0E4FEFEF70AF906F060FD81
:104DF000032246494648FFF747FF2D2403000422BB
:104E00001C7044490130FFF73FFF30230470424DCE
:104E1000424C437083702E3B062220004049EB87B2
:104E2000FEF7B0FA062813D0200006F0A9FC0228ED
:104E300009D00321200006F00BFD8D23E3706E3BAB
:104E4000237119336371062220003549FEF7D4F926
:104E5000344B1B68FC335C64FFF766FF0020FFF7F0
:104E60008FFF314C314A0121314B1278207802F00A
:104E700087F9304A304B12780021207802F080F90F
:104E800001222E4B1A702E4BDB78552B31D12D4B36
:104E90003B325A722C4B2D4AAB81EA812B826A82BB
:104EA0002021307806F034FE0120404205F078FDE4
:104EB0000120404205F014FEFFF720F9FEF7E2FE64
:104EC00000F0A4FC01204042FEF7AAFF012006F0FA
:104ED00017FCF02001F010FB0121307806F098FD5E
:104EE000307802F0E7FA1A4806F042FEFEF7DEFDDF
:104EF00070BD6422174B5B7953431A000A32CBE72B
:104F00005C5CFF1F614B00115D4C0011C43DFF1F35
:104F1000F85BFF1F185CFF1F4E3DFF1F6509FF1F59
:104F2000ADAC0000B05EFF1F865EFF1FA83CFF1FF8
:104F3000893CFF1F5A5EFF1F3B5EFF1F2C5EFF1F59
:104F40003C5CFF1F305CFF1FC4090000CE0900005D
:104F50005E5CFF1F405CFF1FF8B50A0020230D00B8
:104F60001A40194257D0574B1B78002B50D0FFF7EF
:104F7000F1FA554B554C564E99686268737A8A1A05
:104F8000DB039A4202D36160FEF790FD327A217A08
:104F9000531EDBB2994205D1FFF768F9002000F0FB
:104FA000D9FD0FE09142F9D300232372FFF788F96E
:104FB000012000F0CFFD474F3800FEF77FFE39009B
:104FC00006F026FE637A002B1FD0013BDBB2637232
:104FD000002B1AD1404BDB78552B01D106F0E0FDB8
:104FE000E37A002B0CD000233C4A3A4FE37213883B
:104FF000380001331380FEF761FE390006F008FE29
:10500000642370795843FFF7ADFD237A013323728F
:1050100020206840F8BD0BB2002B0ADA304B18781C
:1050200006F086FB002801D006F0D2FC80200002AA
:10503000EFE70224214206D0244B01201A72FFF729
:105040009FFE2000E5E70B071ED5FFF783FA1E4BF6
:105050001E491F4C98684A68637A821ADB039A4299
:1050600002D34860FEF722FDFFF72AF9FFF7FEF8AA
:10507000012000F06FFD00F0E3FB2368DB0701D5A2
:10508000FEF7C6FF0820C4E71024214206D00D4BCE
:105090001B78002BD5D1FEF709FED2E7012421426F
:1050A00007D0104800F06CF806F0B2FA00F034FDBA
:1050B000C7E70424080020402142ABD0FEF7CCFE15
:1050C000BFE7C0465E5EFF1F4C5CFF1F305CFF1FEA
:1050D000405CFF1F893CFF1F3C5CFF1F245CFF1FDF
:1050E0005C5CFF1F6C3CFF1FF0B51B4B1B4F1B880C
:1050F0003A8804001A4E1B4D85B09A420DD832886A
:105100009A420AD3184B1A882B889A4205D1174A1B
:10511000174B12881B889A421BD0052001F042FAD7
:105120003B8802AA13803388019053802B88114D4D
:1051300093800F4B02A91B88D3800F4B2A781888C5
:1051400002F05EFF0D4B08212878019A1C7006F0D2
:105150001FFD05B0F0BDC0462A5EFF1F7E3CFF1F4D
:105160007C3CFF1F7A3CFF1F285EFF1F265EFF1F4F
:10517000783CFF1F865EFF1F803CFF1F245EFF1FE1
:1051800013B50C4B1C78002C11D1002801D00A4B10
:1051900018600A4A0A4B11780A4A10780A4A0192A2
:1051A0000A4A0092002205F0A7FA200016BD112439
:1051B000FBE7C046855EFF1F205EFF1F845EFF1F6A
:1051C000745EFF1F865EFF1F605EFF1F645EFF1F31
:1051D00010B5064B12201B78052B06D1044B132269
:1051E0001988044B187801F0B9FB10BD855EFF1FCC
:1051F000803CFF1F865EFF1F10B500240122114B6B
:1052000052421870104B1C70104B1A8002F052F969
:1052100004220F4B21001A700E480C3206F0E0FAFF
:10522000102221000C4806F0DBFA07220B4B1C6011
:105230000B4B1C700B4B1C700B4B1A700B4B1C70E8
:1052400010BDC046865EFF1F855EFF1F803CFF1FAE
:10525000845EFF1F745EFF1F645EFF1F605EFF1FA2
:105260003A5EFF1F395EFF1F823CFF1F385EFF1F43
:10527000F8B5174C0600257806A814240078052DEB
:1052800023D1B41F134FA5B21824BD421DD88D1FC2
:10529000ADB2BD4219D8FA256D00AA4215D21D0043
:1052A0000D4F0A3DADB2BD420FD80C4C26800C4CC0
:1052B00021800C4900240A800B4A1380FFF714FF59
:1052C0000A4B0421187806F01BFC2000F8BDC046EC
:1052D000855EFF1F790C0000750C00007E3CFF1FEF
:1052E0007C3CFF1F7A3CFF1F783CFF1F865EFF1F40
:1052F000F0B50BB20D0089B0002B00DB70E1A44EBD
:10530000307806F015FA041E50D00378A22B00D195
:1053100022E1D02B1AD0912B45D143780E2B42D1CC
:105320009C4B82889A423ED19B4A83681278052A18
:1053300039D1032018567F2835D0984B1B68002B95
:1053400031D05B68002B2ED098472CE0807807285E
:1053500029D806F045FB0428183F3F74A8D8637885
:10536000002B0CD101218C4B19708D4B1A78002A1F
:105370005BD08C4B307801F003FF002855D007221A
:10538000854B1A7051E061780029F8D1E378002B41
:1053900011D0854A854B1278307801F0F1FE6070AB
:1053A0006378002BEBD1200006F012FB8020000276
:1053B000684009B0F0BD784B1B78022BF3D0012177
:1053C000307806F0C5F90028EAD10121307806F0DE
:1053D0001FFBE5E76378002BD1D16F4F032807D17E
:1053E0003B78052B02D101333B701EE00223FBE723
:1053F0006F4B1A886F4B0293002A0BD01B78002B3F
:1054000003D00121307806F0C3FB3B78062B04D192
:10541000013BE9E7029B1A70F7E7042B41D1012118
:10542000029B3078197006F0F3FA5C4B1B68002B76
:10543000B9D01B68002BB6D0574A107884E7637840
:10544000554F002B27D10622211D5B4806F030FB6B
:1054500062895A4B5A491A80A2895A4B1A80E389A9
:105460000B800521397058490A80584A1380228AD6
:10547000574B1A80574B1B78012B09D11F2001F085
:1054800091F8FA22920042430421307806F080FB22
:105490000022484B75E7312B00D070E70022454BC6
:1054A0001A700323A0E706220021434806F098F96A
:1054B0000023454A04211380444A30781380444A2B
:1054C000138006F01DFB0821307806F019FBA37944
:1054D000083B5A425341304A03331370304B1B7818
:1054E000002B06D0334B30781A78002A06D001F012
:1054F00085FE0122314B52421A8096E70121197034
:1055000006F086FAF5E70821307806F0F9FA6378B4
:10551000002B00D047E72C4B2D4F0293E388029AD3
:1055200004211380294B307803932389039A138035
:1055300063893B8006F00CF9002800D033E7264B46
:105540001B68002B00D12EE7039902983A8809883E
:1055500000881B68984726E74379132B00D022E781
:105560000389012B0AD11D4B1B78022B06D1082180
:10557000307806F0C5FAFFF72BFE14E7052001F09E
:1055800011F808210200307806F002FB0BE7C04654
:10559000865EFF1F05140000855EFF1F205EFF1F53
:1055A000A83CFF1F893CFF1F5A5EFF1F3B5EFF1F89
:1055B0005C5EFF1F5E5EFF1F2D5EFF1F803CFF1FB6
:1055C000345EFF1F365EFF1F2A5EFF1F285EFF1F2F
:1055D000265EFF1F2C5EFF1F1C5EFF1F245EFF1F49
:1055E0008020C001014200D0E2E6CB0731D5324B2A
:1055F0001B78002B1DD0314E05AC3378052B1AD10A
:10560000023B23702E4B21001B7823722D4B1B78FD
:1056100063722D4B187801F057FD002809D0072040
:105620002A4B30701B68002B03D01B68002B00D066
:1056300098470120BCE60E20254B06221B78254901
:105640002370254B1B78637002ABC01806F030FA4C
:10565000D8E7022308001840194209D0174B1B78DD
:10566000052B03D11D4B188806F00AF902209FE68E
:105670000424214203D0FFF737FD200098E60823D9
:1056800008001840194200D193E6154B1C78012CF4
:1056900003D0022C0DD008208AE6124B124A13497F
:1056A00013481B881288098800880094FFF7E0FDE2
:1056B000F1E7FFF78DFDEEE75E5EFF1F855EFF1FE2
:1056C000823CFF1F385EFF1F865EFF1F205EFF1FAC
:1056D0003A5EFF1F833CFF1F395EFF1F803CFF1FA8
:1056E000245EFF1F783CFF1F7A3CFF1F7C3CFF1F9E
:1056F0007E3CFF1F10B502A804880B20002C10D19F
:10570000496808784978090201430C48814209D167
:10571000022119800A4B59881170DB7800205BB296
:10572000537010BD074C0A20A142FAD10221198002
:10573000034B998811705B79F0E7C0466E2A000030
:10574000245CFF1F6F2A0000F7B5150008AA168811
:105750004A680F4F14785278120222430A24BA4240
:1057600014D10122DBB2019200962A0005F0CAFE94
:10577000041E0BD1074B1B68002B07D068782A78D2
:105780000002104342425041013098472000FEBDC4
:1057900002290000985EFF1F30B50125037904003F
:1057A000BFB02B4225D01449408805F017FA284293
:1057B0000CD0124B01A95B8D00220B8002234B8081
:1057C0000F4B5B888B80608802F010FB0D4960886E
:1057D00005F004FAC0070CD50B4B01A91B88002269
:1057E0000B8002234B80064B9B888B80608802F0E5
:1057F000FDFA3FB030BDC046905EFF1FAC3CFF1FBE
:10580000245CFF1F885EFF1F063DFF1F10B5074C7D
:105810000749200005F098F92000064905F094F9A1
:105820000721054A054805F051F910BDFFFF0000AA
:10583000905EFF1F885EFF1F4CBD0011AC3CFF1F38
:1058400010B5024803F054F910BDC0469957001135
:10585000082110B50E240A4AC307DB170B40517903
:10586000A1430B4353710223184202D051790B43D9
:1058700053710423184202D051790B43537110BD68
:105880001D3DFF1F0A2110B50F240A4AC307DB176D
:105890000B401178A1430B431370830703D50623F4
:1058A00011780B431370400703D5012311780B4384
:1058B000137010BD1D3DFF1F10B5054B1024197846
:1058C0000A00A243002801D022000A431A7010BD2A
:1058D0001D3DFF1F662110B52024134BDA788A4343
:1058E0001979DA70A14324190C431C71542812D978
:1058F00060200143197104210A43DA700222D97829
:105900000A43DA702022D9780A43DA704022D97823
:105910000A43DA7007E04428EDD83428EED824286A
:10592000F0D81428F2D810BD1D3DFF1FF8B50E2386
:10593000384C0500627926791A4011339E43364B64
:1059400062712671984204DD6E23E3716C3BA37192
:10595000F8BD324B984203DA1A23E3711C33F6E7A1
:1059600000232F49A371E37183B259182D4889B2DE
:10597000814224D9681D0A2100B205F0F9FE2A4BA4
:1059800000B29D4244DC05006421280005F0F0FED1
:105990000A2100B205F064FE244F09B2E2797B5C73
:1059A0001343E3710A21280005F0E2FE0A2100B248
:1059B00005F056FE1D4F09B27B5CA2790EE0012175
:1059C0000A436271002D1CDA5B421DB20423A371ED
:1059D000A379632DD8DCFA22092DE3DC1343A371EC
:1059E0000A21280005F03CFE0F22114F09B27B5C12
:1059F0001A4016431F229343627926711343637141
:105A0000A6E7FA239B009D42E2DB0123E371BBE79B
:105A10000500FAE71D3DFF1F1B4E00001DFCFFFFA8
:105A2000CB070000960F00000A27000096BD00116A
:105A300086BD001170B51B4D04002B7900290DD0D7
:105A4000802213432B71632C0BDD76236A7813437A
:105A50006B704023AA781343AB7070BD7F22134054
:105A6000F0E72300093306DA58236A7813436B7092
:105A7000AA786C23EFE70C4E002C0ADA202364424C
:105A800024B26B700A21200005F0EAFD09B2735CB4
:105A9000E2E7092CF6DD0A21200005F069FE00B2DC
:105AA000335CEEE71D3DFF1F76BD0011F8B50A4FD0
:105AB00005003B780E00002B0CD0084C2000FEF7B0
:105AC00013FC33002A0020003978FEF701FD200086
:105AD000FEF748FCF8BDC046A55EFF1F283DFF1F2E
:105AE00070B50A4E0A4D08223100280005F080FFEB
:105AF000002809D0074C31000822280005F0D8FF03
:105B000009212000FFF7D2FF70BDC0461D3DFF1FD9
:105B10009D5EFF1F9C5EFF1F102110B50C4B3620B1
:105B20001A7898710A401A70DA7856310A40DA7099
:105B30006022197998701140223ADA71A2325A71B2
:105B4000DF3A0A431A7106225A70FFF7C9FF10BDE7
:105B50001D3DFF1F10B5002824D0134C0A2102233D
:105B6000E05E05F005FE00B2FFF7E0FE0423E05E14
:105B7000642105F0FDFD012100B2FFF75BFF207AF3
:105B8000FFF7A8FE0320FFF763FE0020FFF77AFE71
:105B9000064B1878053843425841C0B2FFF78CFED7
:105BA000FFF79EFF10BDC046245CFF1F855EFF1FF0
:105BB00070B500250A4C2000A571FEF795FB102357
:105BC0003E212000074AFEF783FCA84200D13E3563
:105BD000054B20001D70FEF7C5FB0123A37170BDAE
:105BE000283DFF1F66BD0011A55EFF1F0200F0B536
:105BF00001270A480A4E51188B1A002B00DCF0BD11
:105C0000082415784308684038404000805B013C18
:105C100058406D08002CF5D10132EDE7FFFF000080
:105C2000A6BD0011F0B500250F269D4200DBF0BD9A
:105C30004C5D070944403440A400A0580135784029
:105C4000F3E70000F0B589B06A460D000B000F279E
:105C5000110010351C780133260024093E401670CF
:105C600054700232AB42F5D12023024AFFF7DAFF2B
:105C700009B0F0BDACBD0011F0B54E780B7889B01D
:105C800036020C00170001901E43012A61D9954B82
:105C90009E4200D877E001339E421CD1062A17D1DC
:105CA000CA788B7812021A430B791B0413434A7982
:105CB00012061A438C4B5A6100221A705A808B4A82
:105CC0005A608B4A9A608B4ADA60002009B0F0BDB6
:105CD00088225205EEE7884B9E423CD182498B7860
:105CE000002B00D0F6E00C2A31D10F22A378934389
:105CF000E2781202134322791204134362791206E6
:105D000013434B60E279A07912020243207A000427
:105D10001043627A12060243CA60E27AA07A120243
:105D2000024376484A81834208D804236E491422EC
:105D300001980B7005F0BCFE1420C7E71201D218C1
:105D400089235B059A42F0D801238B70BDE7022AB4
:105D5000FAD00523EAE76A4A01239642E6D1FFF723
:105D600037FA052F0CD9E378A2781B021343227966
:105D700012041A4363791B061343624A03931360A8
:105D800005F00EFFA1E7584D2B78002B9DD1AB7885
:105D9000002B00D1A0E02B8901339BB20093B342CA
:105DA00000D091E0132AD4D9CF7C8B7C3F02122102
:105DB00020001F43FFF71AFF874200D08EE0002E1D
:105DC0003DD1E378A2781B0213432279E9681204DB
:105DD0001A4363791B06134303930A228B4212D1A1
:105DE000FF23A370E370237163716B89002B09D1CA
:105DF000E37B227C1B0212041343A27B13431B0987
:105E000001336B8100226B89002B8ED0002A67D171
:105E1000686837013818000B6B69000303909842DB
:105E200005D9686105F0ECFCEB780133EB7068682C
:105E30001022A11C381805F0BBFE2E8145E76F89A2
:105E4000009A7B1E9BB293423AD1E278A378120269
:105E50001A43237905A81B04134362796C68120660
:105E60001A43EB6800920392211D0C22049305F063
:105E70001FFE0120260004A940421036FFF7E2FE73
:105E8000013F012F17D1009A0B232861824200D0D5
:105E90004CE704221C49200005F08AFE042203A9D5
:105EA000686805F08DFEE968039AFF23914200D1EE
:105EB0003CE7F73B3AE73100FFF7C4FE1036DFE777
:105EC0000923B742A4D831E7009BB34200D9FCE6CE
:105ED00007232BE7022329E7032327E7062325E7E8
:105EE0000A2323E7FFFE0000303DFF1F00000111E1
:105EF000FFFF00005048593601FF0000FFFF00116E
:105F000002FF000034F000403C3DFF1F10B5034C81
:105F10000B000122210000F06BFA10BDCD600011D2
:105F20000B8870B506000D000224162B11D92B002A
:105F30000322094900F05CFA041E0AD1074B2A88A3
:105F40001B88191C934200D9111C300089B200F043
:105F5000EFFA200070BDC046F9600011CA5EFF1F55
:105F600010B54A780400013A0B000220012A07D834
:105F70000A78002A04D005222000024900F038FAED
:105F800010BDC046276100110A7810B50B0004004F
:105F90000220002A04D007222000024900F028FA3B
:105FA00010BDC046D36100110A7810B50B00040083
:105FB0000220002A04D009222000024900F018FA29
:105FC00010BDC0463962001110B5034C0B000B2206
:105FD000210000F00DFA10BD6962001110B5034CEC
:105FE0000B000D22210000F003FA10BDDB6200114E
:105FF00010B5034C0B000F22210000F0F9F910BD81
:10600000356300110A7810B50B0004000220002A45
:1060100004D011222000024900F0EAF910BDC04668
:1060200045630011002310B51322190000F0E0F9B8
:1060300010BD000010B5034C0B001722210000F02A
:10604000D7F910BD97630011002310B5192219006C
:1060500000F0CEF910BD000010B5034C0B001B2260
:10606000210000F0C5F910BDD1630011F7B5848996
:106070000D0006000121002C22D000238268D35697
:106080001778002B1EDA0C2C1AD90C3CA4B2131969
:1060900040880093230002F086FE431E98410130A1
:1060A0007B06DB0F6B703F23013C1F40A4B22870BE
:1060B000AF70AC80002C07D0B3680133AB60002117
:1060C0000800FEBD0020EBE7AC60F8E70B7803703A
:1060D0004B8843704B881B0A83700B79C370042074
:1060E00070470420022B06D10020537811781B0240
:1060F000009A0B43138070470B8803700B881B0AB0
:106100004370022070470420009983420AD15378DB
:1061100010781B0203430B80D37890781B02034353
:1061200000204B807047F8B50D004B78012400210A
:10613000461C03702B788B4201D82000F8BD6B7889
:10614000B01C4F1C012B10D1890069184B8802220A
:1061500033704B88B9001B0A7370691805F080FC16
:1061600004360434A4B2F9B2E4E7122359436B189D
:106170005A88043132705B8810221B0A73706918C8
:1061800005F06EFC12361234ECE770B5049D140075
:106190001E00052B01D8042070BD637812781B0205
:1061A00013432B80E378A2781B02134302226B80F7
:1061B0002A71211D681D063E05F052FCB2B22A81EB
:1061C000E92AE8D82800A11D0A3005F049FC002082
:1061D000E2E7002310B50A789A4201D8900010BD7A
:1061E0009A008A185488013304705488DBB2240A58
:1061F0004470948884709288120AC2700430EAE76E
:1062000010B51100029C062B04D004201022142B80
:1062100001D010BD022222714B7808781B02034383
:106220002380CB7888781B02034363800431601D90
:1062300005F016FC0020ECE710B50C788B780431E3
:106240005C43E4B203702200013005F009FC601CDD
:1062500010BD0420022B06D10020537811781B02B8
:10626000009A0B431380704710B50C000A88023166
:1062700005F0F6FB208810BD70B504000D000498F1
:106280001100012B01D8042070BD1678527812023B
:10629000324302800200F13255701470E125002C67
:1062A00000D10C35023B9AB24280AA42EBD80231AF
:1062B000043005F0D5FB0020E6E704200099834276
:1062C0000AD1537810781B0203430B80D37890785F
:1062D0001B02034300204B80704710B50C000A8856
:1062E000023105F0BDFB208810BD000070B5012112
:1062F0001E000420049C0E400B4218D1CB40DDB29E
:106300008D4214D90A49DBB2098899420FD3230080
:10631000EE331D703300580011184978165C0902DD
:10632000314301332152D9B28D42F4D8002070BDDF
:10633000483DFF1F10B50C000A88023105F090FBA4
:10634000208810BD10B50C788B7804315C43E4B222
:1063500003702200013005F083FB601C10BD10B5F6
:1063600011000298032B01D8042010BD1478527834
:10637000043B120222430280CA788C781202224324
:1063800042809AB28280EB2AEED80431063005F0C2
:1063900067FB0020E9E710B50C000B8803700B8841
:1063A0001B0A43704B8883704B881B0AC3708A8812
:1063B0000430063105F054FBA088043080B210BDD3
:1063C0000420012B03D100201378009A137070472A
:1063D00010B50C000B8803700B881B0A43704A88A9
:1063E0000230043105F03CFB6088023080B210BD01
:1063F000F0B589B003931E4B029242000700D05AB9
:10640000019102F020F81325061E2DD0029B0124D5
:106410000370019B002B04D00019039998470019C1
:1064200084B26B461B7A5BB2002B0FDA1021380066
:1064300002F01CFB1925002813D130003219E1B2FB
:1064400002F066FC051E0CD10C34A4B2042304AA8D
:10645000380005A993800696948101F0AFFD051ED2
:1064600002D0300005F074FB280009B0F0BDC04632
:10647000C85EFF1F70B505000C0000280CD000207E
:10648000814209D010222000044905F0E9FA0120D8
:106490002B7823736B78637370BDC046ECBD00111D
:1064A000F0B506000D0017001C0085B002291BD0B6
:1064B0000020102907D1022B07D0102B03D115E0A3
:1064C0000020102C08D005B0F0BD69463800FFF759
:1064D000D1FF2A0069460BE069463000FFF7CAFF8A
:1064E00022006946380004E0022BE9D12A00390075
:1064F000300005F025FBE6E7031CF02800D9F02367
:10650000032008499AB2013A0B80D3170340064989
:106510009B189B100B80D30F04499B185B100B80BA
:106520007047C0464C3DFF1F4A3DFF1F483DFF1FBF
:10653000034B1B888B4202D3024B4000C152704771
:106540004C3DFF1FC85EFF1F014B4000185A7047AB
:10655000C85EFF1F1722014B1A807047C85EFF1FDD
:1065600070B505000E2005F0E3F9041E13D0D0230A
:10657000037000230622837007494570033005F03D
:106580006FFA064B2100DA8A62811B7E2373044B6B
:10659000187805F095F870BDE45EFF1FD45EFF1F0C
:1065A0009C3DFF1F262803D8024B4000C05A70476D
:1065B0000148FCE74E3DFF1FFFFF000070B50600DD
:1065C0000C00094D1C220021280005F009F9074B99
:1065D0001E70074B1C7005F0F3F90123002801D051
:1065E000002312202B7070BDD45EFF1F9C3DFF1F47
:1065F000F55EFF1F70B505000D4C0800E260A1605C
:1066000010220021656005F013F8012803D1102144
:10661000A06802F058FD10220021280005F008F8BB
:10662000012803D11021606802F04DFD70BDC04605
:10663000D45EFF1F70B5041E05D1002903D00622C9
:106640000D4805F00DFA0D4B1D78012D11D1002CD0
:1066500005D102221A7005F023FA280070BD00222D
:106660001A70074B1B78FF2BF7D02000FFF778FF3D
:10667000F3E70025F1E7C046E45EFF1FD45EFF1F8D
:106680009C3DFF1F030010B5002801D1002010BD64
:1066900000780B4A002803D15988D1821B791376E0
:1066A0001378022BF2D10023984200D103331370E8
:1066B000044B1B78FF2B01D0FFF752FF0120E6E7C8
:1066C000D45EFF1F9C3DFF1F002911D000280CD075
:1066D0004B79012803D140225242134303E03F2269
:1066E0001340032802D001204B7170474022F4E789
:1066F0000800FAE770B5094D0100287800280BD092
:10670000074C0622200005F0ABF921002878FFF79E
:10671000DBFF200004F0DCFF70BDC046F45EFF1F0D
:10672000CE5EFF1F00290AD0012808D13F224B79F5
:106730009343C02B03D0403B5A425341981C7047AF
:1067400070B5174D06002B78FF2B15D00A2005F0E9
:10675000EFF8041E10D0D0230370C83B8370114B98
:1067600011491B784670C3700622043005F078F991
:106770002100287804F0A4FF0C4B1B78012B0DD1CD
:106780000B4B1B68002B03D09B68002B00D0984755
:10679000084B04211878084A05F012F870BDC0466D
:1067A0009C3DFF1FF45EFF1FCE5EFF1FF05EFF1FCC
:1067B0001C5FFF1F205FFF1F60EA0000014B98680D
:1067C0007047C046D45EFF1F014BDB6818687047F6
:1067D000D45EFF1F074B10B5DA68136801331360EE
:1067E000054B1878FF2803D08021C90105F010F966
:1067F00010BDC046D45EFF1F9C3DFF1FF7B50E00C5
:1068000002F0C8F8051E1CD00E4B06621F78002F40
:1068100000D10778AB791020019305F089F8041EA8
:106820000FD0D0230380C73B8370019BE91DC37049
:106830000622043005F014F921003800E66004F067
:106840003FFFF7BD9A3DFF1F014B18787047C046C8
:10685000F45EFF1F054B002805D1054B1A78054B48
:10686000002A00D1014B18007047C046E45EFF1FAC
:10687000F45EFF1FCE5EFF1F014B58687047C04695
:10688000D45EFF1F024B1868431E9841C0B2704788
:10689000F85EFF1F421E03000120152A03D9FF3BAB
:1068A0005A425341D8B27047F0B51C0000230E0085
:1068B00085B0039002920B70029A934201D300209C
:1068C00019E0E55C5A1CD2B2002DF8D0029851199B
:1068D0008142F4DC0233DFB2A35C18000193FFF7BE
:1068E000D9FF002807D0013D019A0399EBB233701C
:1068F0008A4202D1E01905B0F0BDDB19DBB2DBE75B
:1069000010B50C0002F09EF803001220002B03D0FB
:106910002100588804F0FCFE10BD000070B50E4D3B
:1069200084006359002B15D0186A002801D004F0A8
:10693000D7FE2B59586A002801D004F0D1FE2B59FC
:10694000986A002801D004F0CBFE285904F0C8FE54
:1069500000232B5170BDC046045FFF1F1C4B70B558
:1069600004000E00150099420AD11A4B1B68002B37
:1069700001D1122070BD1B68002BFAD09847F9E7AF
:10698000154B994215D1134B1B68002B0AD01B687D
:10699000002B07D09847002804D1104B1C70104BD7
:1069A0001D70E7E729002000FFF7AAFF0028E1D1CA
:1069B000F3E7080001F0EEFF0028DAD003780320A7
:1069C000A342D7D12900300004F0A2FED2E7C0468E
:1069D000FEFF0000005FFF1FFFFF0000FD5EFF1FC6
:1069E000FC5EFF1FF7B50400808801F0D3FF00258F
:1069F000A84203D00578A08802F008F81C4E33782E
:106A0000002B1FD0AB421DD11A4B28001978FFF77D
:106A100077FF002818D000233370A3790820A778C7
:106A2000A688019304F084FF011E0DD0D0230370CB
:106A3000CA3B8370019B477086808371280004F0F5
:106A40003FFE01E0002DE8D1A0880B4B8200D35817
:106A5000002B01D0FFF762FF1721A088FFF768FD28
:106A6000A08801F027FDA08801F0FEFDF7BDC0461B
:106A7000FD5EFF1FFC5EFF1F045FFF1FF0B587B0C8
:106A80001D000CAB1B88070001930DAB1B88142065
:106A900002930EAB1B88160003930FAB1B8800916B
:106AA000049310AB1B88059304F042FF041E1AD018
:106AB000D0230370CB3B47708370C6700622290039
:106AC0000430002D11D004F0CBFF019B2100638125
:106AD000029B0098A381039BE381049B2382059B77
:106AE000A37404F0EDFD07B0F0BD04F079FEECE70F
:106AF000F7B5009308AB1B8807000C200D001600AB
:106B0000019304F015FF041E13D0280001F042FF8A
:106B100000280FD00078D0232370C93BA370009BBE
:106B200021002381019B6770A580E680638104F0CA
:106B3000C7FDF7BD014B1878EDE7C0469C3DFF1F30
:106B400013B5040064890389C2888188C0780094E1
:106B5000FFF7CEFF13BD000010B5044C20680028DD
:106B600003D004F0BDFD0023236010BD085FFF1FAC
:106B7000A122F0B5818892004A43384B384F1B68F8
:106B800004009B189D2292009B18827989B01A609C
:106B90003B68002B5FD01D78324B1B68002B04D064
:106BA0005B68002B01D00020984726000836310092
:106BB000E079FFF7B7FD237DE0710200E0780493F0
:106BC000638A29000393238A0293E3890193A388AC
:106BD00000933300FFF752FFE378002B0BD1E289DB
:106BE000A379A18802920196E279280000920122FD
:106BF00001F0DAFEE0703B68002B20D0FFF7ACFF1D
:106C0000194D287800281AD0184B1978FFF778FE0C
:106C1000002814D02B78E67808200793A78804F082
:106C200087FE011E09D0D0230370CA3B46708370D3
:106C300087808671079804F043FD00232B7017218D
:106C4000A088FFF775FCA08801F034FCA08801F053
:106C50000BFD09B0F0BD064B9DE7C0463409FF1F90
:106C6000085FFF1F1C5FFF1FFD5EFF1FFC5EFF1F15
:106C70009C3DFF1FF8B5070008000E0001F08AFEDA
:106C8000041E18D02620FFF78DFC051E00D12578A4
:106C9000062004F04DFE041E0DD00021062204F053
:106CA0009FFDD0232370C23B21006770A370A68094
:106CB000E8B204F005FDF8BDF0B585B001930AAB6C
:106CC0001B78070002930BAB1B7808000D000092A5
:106CD000039301F05FFE061E22D0102004F028FE70
:106CE000041E1DD01022002104F07AFD2620FFF79B
:106CF00059FC002800D13078D0232370C13BA37009
:106D0000009B21002372019B67706372029BA58028
:106D1000A372039BC0B2E3720C9BE36004F0D0FC4F
:106D200005B0F0BDF7B50D00019001F033FE071E70
:106D300020D00E2004F0FCFD041E1BD02620FFF7FF
:106D400031FC061E00D13E78D0232380C53B0622AD
:106D5000A370F91DE01C04F083FE019B2A006381EF
:106D60000123DD401A401D40210022736573F0B2FB
:106D700004F0A6FCF7BD0000F0B585B0029010004D
:106D80000D0017000A9E039301F004FE041E31D08B
:106D9000029B002B2ED1039B02795B0724D5122383
:106DA00013430422002E08D10B99002905D10C9918
:106DB000002902D10D9900291AD01A430D9B227186
:106DC000002B00D0C9E0002E00D1CFE0002D00D074
:106DD000CCE0606A002801D004F082FC1C21300065
:106DE00004F0E6FD606205E002239A430E33D7E724
:106DF00093432371654BBA00D458002C00D1AAE00C
:106E0000002E10D0236A002B03D11C2004F088FD33
:106E100020625E4BBA00D358186A002803D01C22A7
:106E2000310004F01DFE0C9B002B12D0574CBB0010
:106E30001D596B6A002B03D1162004F071FD6862A6
:106E4000BB00E358586A002803D016220C9904F0BE
:106E500007FE0D9B002B11D04C4DBC006659B36A48
:106E6000002B03D1142004F05BFDB0622B59986A0B
:106E7000002803D014220D9904F0F2FD380001F02F
:106E800089FD051E67D0414BBA00D358002B62D054
:106E90001A6A3420002A00D11C389A6A002A01D0CC
:106EA000143080B20B9A002A01D01C3080B25B6A89
:106EB000002B01D0163080B204F03AFD041E4AD0F7
:106EC0001822002104F08CFC2620FFF76BFB0190B8
:106ED000002801D12B780193D0232370029B20003E
:106EE00063700A23294EA370039BBD00A371AB59A5
:106EF000A780196A1830002905D01C22A06004F070
:106F0000AFFD200034307359996A002907D003007F
:106F100014221433E060029304F0A2FD02980B9B4C
:106F2000002B08D003001C221C330B992061029314
:106F300004F096FD02987359596A002903D016226D
:106F4000606104F08DFD6B462100187904F0B8FBF8
:106F50003800FFF7E3FC05B0F0BD10220D9B0D9942
:106F60001B69A018236204F07BFD2CE70B9B002B10
:106F700000D13FE7012D00D03CE7606A002801D036
:106F800004F0AEFB1C210B982AE7C046045FFF1FEC
:106F900010B5044C2068002803D004F0A1FB0023A6
:106FA000236010BDF85EFF1F0B4B07B51A68002A5F
:106FB00001D100200EBD6946531C01201278073113
:106FC000FFF772FC0028F4D002780123100018406B
:106FD0001A42EED0EEE7C046145FFF1FF0B51F4F18
:106FE00001203B6887B0002B25D09B78059300F0EB
:106FF000B3FB002821D00A20FFF7D4FA04000B20AD
:10700000FFF7D0FA164B05001E78731E9E413B68B1
:10701000F6B2191DD878FFF757FB3B682900DA7ADA
:10702000043303929A790193029200903300200076
:10703000059A04F005FD07B0F0BDFFF7B5FF002885
:1070400005D00620FFF7AEFA04000720D8E7082095
:10705000FFF7A8FA04000920D2E7C046F85EFF1F38
:10706000F45EFF1F70B50A4E040033780D00FF2B4D
:107070000DD0042004F05CFC011E08D0D023037066
:10708000CE3B45708370C470307804F019FB70BD3E
:10709000AC3DFF1F70B5040006200D0004F048FC55
:1070A000011E0AD0D0230370CD3B8370054B447082
:1070B0001B688580187804F003FB002C01D0FFF7D3
:1070C00067FF70BDF85EFF1FF8B5264F06003B68EE
:1070D0000D001124002B05D10522234B1B781342F0
:1070E00002D112242000F8BD204A10241268002A80
:1070F000F8D01278002AF5D0DB0719D52B789A1E24
:10710000012A1AD80C2004F00BFC13243860002844
:10711000E8D000230A22437029000670023004F0F0
:107120009FFCFFF75BFF041E0AD0FFF731FFD9E792
:1071300000F012FB0028E1D1E4E7002BE2D0D0E719
:107140000B4B1B78032BCDD11D20FFF72BFA094BDE
:1071500018800028C6D0084B04211878074A04F08C
:107160002FFBBFE7F85EFF1FF55EFF1F145FFF1FD9
:10717000F45EFF1FF25EFF1F205FFF1F60EA00004A
:10718000F7B50193194B14001A78052306000F0078
:1071900012201A4221D0012920D1154B1D68002D43
:1071A0001BD002201F2C18D8002C02D0019B002BD2
:1071B00013D0104B1F221E706E1C0021300004F0F3
:1071C0000FFB01992200300004F04AFC310020003E
:1071D0002C70002F06D004F03BFCFEBD064B1220A5
:1071E0001D68DCE704F0F4FCF7E7C046F55EFF1F1E
:1071F000145FFF1FAC3DFF1F105FFF1FF8B50F4E60
:1072000012243368002B17D01B780F3C834213D114
:1072100000250B4F0221387804F072FC094B042141
:1072200038781D8004F06CFC074B28001D80336803
:107230005C7004F035FA04002000F8BDF85EFF1F12
:10724000205FFF1F0C5FFF1FF25EFF1F70B501285C
:1072500023D11B4C2388002B03D01A4A1578002D0C
:1072600007D0194B1B68002B02D01878FFF7C6FF18
:1072700070BD3B2B02D93C3B2380F9E7134E022122
:10728000307804F03DFCFA222388920002215A4310
:10729000307804F07DFC2580EAE70B4B1B68002B5F
:1072A000E6D00B4B1B785B07E2D5084B0221187820
:1072B00004F026FC0022024B1A80FFF769FED7E794
:1072C0000C5FFF1FF05EFF1FF85EFF1F205FFF1FB8
:1072D000F55EFF1FF8B51E4D2868002803D004F0A6
:1072E000FFF900232B601B4E3068002803D004F008
:1072F000F7F900233360184F05243B78180020402D
:10730000234221D0154800F02BFA3B78234213D0BA
:10731000202004F005FB2860002813D02022002143
:1073200004F05EFA202004F0FBFA041E306005D061
:107330002022002104F054FA002004E0286804F020
:10734000CFF92C601320F8BD00F00AFAF4E7C0462C
:10735000145FFF1F105FFF1FF55EFF1FA03DFF1FA3
:1073600010B50A4C23681A1E0ED0002808D101302F
:10737000587004F095F9002805D02368002B02D03E
:107380000021FFF787FE0122100010BDF85EFF1FED
:10739000F7B5274E050033680191181E21D05C789F
:1073A000244F012C30D1FFF7FFFD002825D020000D
:1073B000FFF7F8F80400412814D91F4B0221187870
:1073C0001E4A04F0FDF91E4B3C3C1C80022233682F
:1073D0005A703B78002B14D128000199FFF75AFE10
:1073E0000120FEBDFA2292004243002AEED0124B49
:1073F0000221187804F0CCFBE8E7FFF7D3F802008D
:10740000F3E700233B70EBE73B78002BE8D1032048
:1074100004F08EFA011E08D0D0230370CC3B4570D7
:1074200083703368187804F04BF9FFF7B1FDD7E7A4
:10743000F85EFF1FF05EFF1F205FFF1F60EA000085
:107440000C5FFF1F10B51749838802008B4220D0C4
:1074500011D815498B4217D0144900205B1899B2F6
:10746000012907D8926811785A425341D8B2FFF7E0
:10747000F9FD012010BD0E4A00209B1807229BB287
:107480009A424041C0B2F5E783681878FFF768FF79
:10749000F0E7836899785A78090218781143FFF762
:1074A00077FFE7E70A20000006200000F8DFFFFF73
:1074B000AFDFFFFF014B18707047C046AD3DFF1FA7
:1074C00010B5064C207001F041FA207804F060F904
:1074D0000521207800F062FD10BDC046205FFF1F2F
:1074E0000BB273B50D00002B00DBC4E0884B18789D
:1074F00004F01EF9041E0ED00378912B0FD0A22B9E
:1075000000D1A1E0834B1878FF2852D0210004F06D
:10751000D7F800284DD180200002684076BD43781E
:107520000F2B76D013D8052B70D00E2BEAD1808884
:10753000794B98422BD8794B98421BD8784B98427C
:10754000E0D1A3681878591CFFF774F838E03E2B97
:10755000D8D18378032B74D06CD8012B6ED0022B3A
:10756000D0D1704B1B68002B23D05B68002B20D040
:1075700098471EE06C4BC0180C28C3D804F038F8AC
:107580001DC2C2150BC20B0B0B3223C23C00674B52
:10759000C0180728B6D8664B1B68002B09D01B689B
:1075A000002B06D0200098470AE0A3681878FFF760
:1075B000C7F8200004F00CFAADE7A068FFF762F806
:1075C00000289FD0F5E7A3681B78002BF1D0554B1E
:1075D0001B68002BEDD01B68002BEAD0210055481A
:1075E0009847EDE74F4B1B68002BE2D01B68002B40
:1075F000DFD021005048F3E7504B1B68002BD8D058
:107600005B68002BD5D021004348E9E7FFF7EAF992
:10761000CFE780884A4B984203D04A4B984200D02B
:1076200070E7464B1B68002BC3D05B68002BC0D0B3
:107630002100D5E7153B012BBBD963E7FFF798FA8B
:10764000B7E7FFF77DFAB4E73F4B1B78042B07D170
:1076500000236A4613800179408800F0C5FCA8E742
:10766000364B1B68002BA4D05B68002BA1D0010017
:10767000364898479DE7012421420AD0294B1B68D0
:10768000002B04D05B68002B01D00020984701201C
:1076900043E78B070AD5264B1B68002B04D05B6899
:1076A000002B01D020009847022036E70421280053
:1076B00008400D4200D131E7254E3388002B21D000
:1076C000013B9BB23380002B1AD1FFF7DBF8002877
:1076D0000AD0204B1C70164B1B68002B04D05B6833
:1076E000002B01D020009847FFF7C6F8694601F04B
:1076F00001FD6846FEF7FEFF1D20FEF753FF3080B8
:1077000004200AE7024B187804F0FAF9F8E7C046BB
:10771000205FFF1FAD3DFF1F0E2000000120000075
:1077200009100000185FFF1FFEDFFFFFAFDFFFFF44
:107730001C5FFF1F0C2000000B200000005FFF1FDC
:107740000D20000013200000F55EFF1FFFFF00006A
:10775000F25EFF1FF05EFF1F10B501F09BF910BD38
:10776000014B18607047C0461C5FFF1F0B8800204C
:10777000162B01D817230420014A13807047C046F6
:10778000CA5EFF1F00207047074A0300118881422C
:1077900007D091880020994202D101308000101852
:1077A00070470020FAE7C046285FFF1FF0B58F78CA
:1077B00006000D00C5B01E2F15D1FFF7E5FF051E11
:1077C00003D10024200045B0F0BD00223B00310071
:1077D000C078009200F0B2FB0400A81C00F0D2FBBD
:1077E000FF23EB70EEE7264B062403931B78FF2B59
:1077F000E8D0182FE6D87B08224A013BDB00029232
:107800009A589446002ADDD0029AD3185B68002B60
:10781000D8D00878002802D14B78012B02D1062459
:10782000122FCFD107AFAB88697800976446AA685A
:10783000A047041EC6D1AB78029A5B08013BDB006F
:10784000D318390030005B689847041E0BD1AB7821
:10785000042BB6D0039A310010782200009700F074
:107860006DFB0400AEE76A78002AABD1AA7805A9BF
:107870003B88087130000A704B80FEF747FBA0E799
:10788000B03DFF1FFCBD00111D4B37B505009842F0
:107890000BD000290AD1FFF777FF002805D119483E
:1078A000FFF772FF002800D0058037BD01291AD1EB
:1078B000FFF76AFF041EF8D001235B420380A37820
:1078C000FF2BF2D0FE2B07D00023E0781422009388
:1078D00029001E3300F032FBA01C00F053FB0123F3
:1078E0005B426380E1E70229DFD1013901F0BEF894
:1078F0000028DAD12800FFF747FF041EDFD1D4E7C4
:10790000FEFF0000FFFF0000022210B5074B5242AD
:107910001A80074801325A809A80DA8000F07EFA95
:10792000044801F025F8002010BDC046285FFF1F65
:10793000AD770011897800110388F7B50400002B9A
:1079400002D102252800FEBD426802211378254895
:107950005268FEF7A5FD00282ED0234F01253A8856
:10796000002AEFD0802321885B0201259B1A9942CF
:10797000E8DC0C2003F0D4FF061E31D03B882288BF
:107980009C4600231800019561469DB2491989B2B1
:10799000AA421BD8002801D062443A80002330005C
:1079A000082208C0210004F05BF8104A1368002B7D
:1079B00013D100251660C5E76268022113780C48D0
:1079C0005268FEF76DFD0028C7D1BAE760681D0157
:1079D0004019418101330198D6E71A001B68E6E798
:1079E0001325AFE76ABE0011AE3DFF1F245FFF1FE6
:1079F00068BE0011014B18707047C046B03DFF1FB4
:107A000014230A0010B51A40194204D00122102193
:107A100001F048F810BD4B06F9D40120884340001E
:107A2000F8E710B514008B0604D50122102101F0EF
:107A300039F810BD08230A001A40194202D14BB28E
:107A4000002B0FDA102101F02DF8002808D02300B8
:107A5000F2331B78002BECD0F1342378012BE8D1E2
:107A60000020E6E703208907FAD4E2E7F0B51F001B
:107A7000184B85B01C68019002910392002C27D10D
:107A8000200005B0F0BDA5683301ED186B89019A9F
:107A9000934211D3029A93420ED8002F04D10A9B2D
:107AA000002B10D12C00EBE73B002978039A686883
:107AB000FEF7F6FC0028F2D10136B6B2A388B34235
:107AC000E1D82468DAE7A3680A9A5B891380E9E7BA
:107AD0000026F3E7245FFF1F37B50C000A884988AA
:107AE0000123914217D3002A15D0651D23792A005E
:107AF00002210A48FEF7D4FC102300280BD023797A
:107B00006188208800242A000094FFF7AFFF0A2331
:107B1000A04200D0230018003EBDC0466ABE00113E
:107B200013B50A0008884988012388420BD8002829
:107B300009D00024137905320094FFF797FF0A2338
:107B4000A04200D02300180016BD13B50A00088813
:107B50004988012388420BD8002809D000241379D2
:107B600005320094FFF782FF0A23A04200D02300D1
:107B7000180016BDF0B58BB003904A8808880E0037
:107B80000123824255D3002853D00023012704AC9F
:107B900023700022718813000092FFF767FF051E13
:107BA0003ED02078002835D12B78022B18D1677071
:107BB0006A8983000130E31880005A8069680222D4
:107BC000201803F04DFF23780133DBB22370042B20
:107BD00019D93B006889013080B2002BD9D01FE051
:107BE00002236370122358436A89231804305A8091
:107BF00069681022201803F033FF23780133DBB2C9
:107C00002370002BE5D10C4A6B899B185A425341D3
:107C1000DBB2DFE76378012BE4D12B78022BC7D0EE
:107C200022780A23002A04D021000398FEF798F94D
:107C3000002318000BB0F0BD0100FFFF0F4BF0B5A3
:107C400004001868002816D083685D89A54207D80B
:107C50008288AE18B44203DA12019A18934201D115
:107C60000068EFE71E005F891036A74204D10029A3
:107C700000D00D801800F0BD3300EFE7245FFF1F38
:107C800070B505000C0008880021FFF7D7FF03003E
:107C90000120002B04D022002800197AFFF7C1FE32
:107CA00070BDF7B50C00002501902300EE331B7862
:107CB000AB4201D800200AE06B00E65A00213000F8
:107CC000E718FFF7BBFF002802D126800130FEBD78
:107CD000017A0198FFF794FE002802D03B882380A8
:107CE000F5E70135EDB2E0E710B5040008880021A2
:107CF000FFF7A4FF03000120002B03D02000197A16
:107D0000FFF77EFE10BD0000054B1B68002B01D164
:107D1000180004E09A6852898242F6D19888704728
:107D2000245FFF1FF0B50E27002687B0039302AB38
:107D3000FF183E8005001F4B40891400984207D071
:107D40002B78013000976A6880B2FFF78FFE06003B
:107D500002212B7818486A68FEF7A2FB00280FD092
:107D60006C892000FFF7D0FF002802D0013C0419E5
:107D7000A4B2039B002B00D01C80300007B0F0BDE4
:107D800002212B780D486A68FEF78AFB0028E7D1AC
:107D900002212B780A486A68FEF782FB002807D088
:107DA000002EDED03B88A342DBD17489013CDFE7A3
:107DB0006C89DEE7FFFF00006ABE001168BE00119B
:107DC00066BE001110B50C00FFF7DEFC03000220B8
:107DD000002B0AD0002C00D023609B781720FE2BAC
:107DE00003D00138FF2B00D1002010BD73B50D006A
:107DF00001A904001600FFF7E5FF172805D0002EA3
:107E000004D129002000FEF727F976BD01221021B8
:107E1000200000F047FE0028F3D0F6E7014B186081
:107E20007047C046345FFF1F37B56B469D1D01008C
:107E300004000222280003F03BFE2B88B02B0ED159
:107E40002379122B09D12300FA331B78012B06D199
:107E50000121608800F0E0F801E01B2BF8D037BD6D
:107E600010B5054B0421187000F098F8FFF74CFD91
:107E7000FEF770FB10BDC046385FFF1F0020F0B555
:107E80000BB20F0087B0834234DA274B187803F027
:107E90004FFC051E2BD00378A02B25D103AE31005B
:107EA000FEF7E4F8041E0BD1B378DB0724D51F4B93
:107EB00006341B68002B03D0310068889847040003
:107EC000A868002801D003F043FE002C08D1184A0E
:107ED000039B1340174A934206D0B3781B2B03D061
:107EE0000121688800F098F8280003F071FD8020D7
:107EF0000002784007B0F0BD0F4B1B68002B10D07C
:107F0000310068889847041EDAD07378002BD7D1E7
:107F1000B27801A90A704B800C716888FDF7F6FFF2
:107F2000CEE70624F1E7C046385FFF1F305FFF1F32
:107F300000FFFF0000011200345FFF1FF7B5019042
:107F4000FC200D0017001E0003F0F2FC04001320BB
:107F5000002C12D0B02320002370089BF4226770FD
:107F6000658026710830002B08D0190003F078FDD9
:107F70002100019803F0A4FB0020FEBD089903F046
:107F80002FFCF5E710B5041E06D00078FD2803D8B5
:107F900003F00EFCFF23237010BD00000A1F93B2F4
:107FA00010B504000220032B05D882400020024BAC
:107FB000D1529B189C7010BD585FFF1F0B8870B585
:107FC000043B04000D000220032B0BD801212000EC
:107FD00000F04CFD03001420002B03D029002000EA
:107FE00000F0DEFB70BD000007B51300034A0092ED
:107FF0000A00012100F02CFC0EBDC04625820011B4
:1080000007B5019203220092024B0A00122100F0F0
:1080100049FC0EBDA382001107B56B4601AA118071
:108020000449D88008780633012802D1190003F0EA
:108030006FFC07BD395FFF1F0C4B10B51870002394
:10804000FF210B4A1380138193819380094A538047
:108050001370517293819372D174D38213755177D7
:1080600003F016FB00F0FCF910BDC046685FFF1F6F
:10807000585FFF1F3A5FFF1FF0B58DB06B460020C1
:1080800003910C229B5E834200DBB0E05D4B1878CD
:1080900003F04EFB051E00D1A4E00378902B00D026
:1080A0009DE006AF01004688380000F013FA7968B9
:1080B0000400002900D19CE03B88052B6ED13B8950
:1080C000032B1CD905AC200000F0A2F86288172A07
:1080D00061D83989131D994231D1796823780431E7
:1080E0000291D90738D5607800F08EF9071E06D0C6
:1080F000002303712378012B08D0132B23D0A86809
:10810000002800D178E003F023FD75E06288029931
:1081100009A800F0A6F80290380000F08BF909AA2F
:108120002378387A0192002231000092029A00F0FE
:1081300012F9380000F064F9029B002BDFD0300008
:1081400000F080F9DBE70378032BD8D1628802992D
:1081500009A800F0D6F8DEE7122B13D1029909A87E
:1081600000F0B5F8021EEAD127498B88002BC6D053
:10817000887909A92378019161780091310000F094
:10818000EAF8BCE7002302AA93833000617809AAC9
:10819000FFF72AFFB3E71D4B0993F6E7042B02D044
:1081A0009A1F012AABD8184A043B9B00995A002910
:1081B000A5D0D218907831003A0000F0AEF800282F
:1081C0009DD13B88042B03D001213000FFF724FF11
:1081D000012C04D1A868002801D003F0B9FC2800C4
:1081E00003F0F6FB8020039B0002434018000DB013
:1081F000F0BD012800D182E701213000FFF70CFF1C
:10820000EDE7C046685FFF1F585FFF1F01001700C2
:108210000B7803704B784370CB788A781B0213433A
:10822000438070470A88030002700A88120A42706D
:108230000A88012A06D14A8882704A88120AC270C6
:108240000420704702208242FBD14A8804309A7091
:108250004A88120ADA708A881A718A88120A5A7150
:10826000EFE710B50400012082420CD94B780A7860
:108270001B0213432380834206D1CB788A781B02EA
:1082800013436380002010BD022BFBD1CB788A788A
:108290001B02134363804B790A791B021343A380AB
:1082A000F0E70B8803700B881B0A43704B888370C0
:1082B0004B881B0AC3708B8803718B881B0A437120
:1082C000CB888371CB881B0AC371082070470300D9
:1082D0000120082A14D14A780878120202431A8031
:1082E000CA788878120202435A804A7908791202C1
:1082F00002439A80CA798879120202430020DA8008
:10830000704710B504000120022A05D100204B78E7
:108310000A781B021343238010BDF8B50600102015
:108320000F00150003F004FB04000120002C0ED008
:10833000A0230C22290023806780201D002D07D058
:1083400003F08EFB2100300003F0BAF90020F8BDE5
:1083500003F046FAF6E7F7B51E00009008AB1420CC
:1083600017001D78019103F0E3FA041E12D0A22336
:108370000370019B47704380099B057146710C2275
:108380000830002B07D0190003F06AFB2100009889
:1083900003F096F9F7BD099903F022FAF6E737B52D
:1083A000041E0FD04388002B0CD00025C188132356
:1083B000007A172201950095FFF7CDFFFF23658016
:1083C0006372257037BD000010B50C4904004A885F
:1083D000002A09D08B89002B05D00020CB8A0222ED
:1083E000834201D010BD012213000A204343002024
:1083F0004032C854C81842800472F3E73A5FFF1F46
:108400000023438003707047094B00211A0010B508
:108410005C88002C06D01C79844203D10A234B438C
:10842000D01810BD01310A330329F1D10020F8E73B
:108430003A5FFF1F10B50400407A03F0B9F9FF233B
:10844000637210BD7047043010B580B203F0A0FA1B
:10845000002803D00421494203F02AF910BD00008E
:1084600070B50025104CA0682580A581A580A84284
:1084700002D003F06DFBA56000250C4C0C4B606D29
:108480001D80230058331D70A84202D003F060FB0A
:10849000656500256068002801D003F059FB0135AF
:1084A00008340A2DF6D170BD0060FF1FA45FFF1FC6
:1084B000F45FFF1F70B5041E09D1054D2880A88107
:1084C000A880A868002802D003F042FBAC6070BD11
:1084D0000060FF1FF0B54B8885B001930023436017
:1084E0000A7905000F00022A00D07BE0CA88032A1F
:1084F00017D98B685E7819783602DC78D8790E4304
:1085000099781B7A24021B020C43034353495BBA3C
:108510000B80331D93421ED1042C04D0631F022B09
:108520000ED9012015E0019A4D4B1201D35A002BB0
:1085300006D00198FFF7BEFF4A4A13690133136161
:108540000421B8682E812C80494203F0B1F868609C
:10855000002005B0F0BD434D042C06D0631F022B54
:108560000FD9EB680133EB60DBE7019A3C4B12015A
:10857000D35A002B05D00198FFF79CFF2B690133DC
:108580002B61374B30000293019B029A1B01019330
:10859000002301998C468B52130063449C80039303
:1085A0009E81FFF750FF039B041E986016D00421A4
:1085B000B868494203F07CF8FA880100043A2000C8
:1085C00003F04EFA0199029AFB888A5A043B9B18E1
:1085D000029A8B522B6801332B60A2E7AB690133FF
:1085E000AB619EE71E4B0293019B1E01029BF35A57
:1085F000002B2DD002998C19A068002828D0012AC0
:1086000026D1FA889B189BB27352A189994217D33D
:108610009B1AC018B96803F023FA029BA289F35A87
:10862000934200D07DE700222B81A3882B80A36892
:108630006B60029BF2520B4A53680133536070E740
:10864000084A9368013393600198FFF733FF68E7A6
:10865000044A536901335361F6E7C0466A5FFF1F5E
:108660000060FF1F705FFF1F70B5051E15D10B4C1A
:108670000B4B1880230058331870606D002802D00F
:1086800003F066FA6565250050356068002801D062
:1086900003F05EFA0834AC42F7D170BDA45FFF1F4F
:1086A000F45FFF1FF0B51700A12285B0920001937F
:1086B0004243394B06001B680C009B18D933FF332B
:1086C0001D78FDF741FF0430854204DD3000FDF7E1
:1086D0003BFF0430C5B2BD4207D33A000021300051
:1086E000019B03F0A5F905B0F0BD2900380003F0A7
:1086F000E7F92300C6B250331E700393019B290093
:108700006365380002F0BCFFCBB20293002B02D0AD
:10871000039B01361E7000262300503303931B7801
:10872000B34204D8606D002831D10020DBE7029A03
:108730002800002A04D0013B1000B34200D02800DA
:10874000F700E719387003F05BFA786000280ED064
:108750003A78019903F084F9019A3B780136D318ED
:108760000E4A0193D369F6B20133D361D4E7039B78
:1087700018706065A74205D1084A1320D36A0133F7
:10878000D362B0E7606803F0E3F90834F2E703F07E
:10879000DFF900236365C8E73409FF1F705FFF1F1F
:1087A000F7B50D0007000421686802F081FF2B89EE
:1087B000040003702B891B0A43702B8883702B885D
:1087C0001B0AC3702E8902250436F6B2F42E15D882
:1087D0001B4B9F4214D10C2003F0AAF81135011E47
:1087E0000CD0902303708E3B0371043B4380154BE8
:1087F0008460C680187802F063FF00252800FEBD63
:108800005C237B43104AD3180093583301931B78A1
:10881000002B0FD10300320038000099FFF742FF10
:10882000019B05001B78002BE8D13800009903F06C
:108830002FF9E3E7054A0725536A01335362DDE761
:10884000FEFF0000685FFF1FA45FFF1F705FFF1F38
:10885000F0B587B0009017200F0016000193FFF7C6
:10886000F2FD1325041E19D00C98031E02D00199A5
:10887000201D9847030AE370052302AAA070043064
:10888000908127700098667003A993800494FFF785
:1088900087FF051E02D0200003F05AF9280007B018
:1088A000F0BD0000F0B587B01F000CAB1B78039142
:1088B000059301210DAB06001C78049200F0D6F858
:1088C0001425002821D02000FFF77EFD0135041E6D
:1088D0001BD01149059B0A7803700132D2B2131ED6
:1088E000C68001D101231A000B7022713000049B55
:1088F00003990097FFF7ACFF051E09D12300210063
:108900000648074A093302F0ABFF280007B0F0BD64
:10891000002363802370F8E76C5FFF1F9F830011C3
:1089200030750000F8B505000E00064C064F2368B0
:10893000002B02D03100280098470434BC42F6D105
:10894000F8BDC0461060FF1F2460FF1F0123064AC8
:108950005B425380002313715362044A13605360D7
:108960009360D360136170472460FF1F1060FF1F86
:108970000200002310B506499C000859002801D1C7
:10898000625010BD0133052BF6D11320F9E7C04624
:108990001060FF1F034A5388181A4342584140424F
:1089A000104070472460FF1FF0B585B002930AABFA
:1089B0001F780CAB1B88009008000E0001920393F7
:1089C000FFF7E8FF05001120002D1BD10E48FFF72F
:1089D000E1FF04001520002C14D006220B99A7718A
:1089E000E01D03F03DF8019B30002371029B29003C
:1089F0006371009B66802370039B6562E381FFF7D0
:108A000091FF280005B0F0BDFFFF000010B5FFF793
:108A1000C1FF04000220002C12D060880121FFF762
:108A200081FF606A002801D002F05AFE282200214E
:108A3000200002F0D5FE012300205B4263802071FC
:108A400010BD000030B5074A074C55880100137867
:108A50000020A54204D05B1A59424B4158421040B5
:108A600030BDC0462460FF1FFFFF0000084A10B55C
:108A700001230C00904208D0FFF78CFF031E04D0A6
:108A8000037923405A1E9341DBB2180010BDC04643
:108A9000FEFF0000024B1879431E9841C0B2704798
:108AA0002460FF1F70B504000D001600FFF772FF71
:108AB000002804D10D4B9C4200D0143070BD416A97
:108AC00003790520002907D012221A40102A02D16A
:108AD0000520002EF2D10F20DB06EFD5897E0C2079
:108AE000A9428941494249420840E7E7FEFF0000A8
:108AF000030010B5002800D110BD0348034A418887
:108B00009142F9D09847F7E72460FF1FFFFF00006C
:108B1000002330B5C45CCD5C6C40D4540133102BC1
:108B2000F8D130BD0F23002210B5C45C640022438D
:108B3000CA54C25CD209013BF7D210BD0200010049
:108B400010B52032103102F00BFF10BDF0B58BB024
:108B50000390102005931700049102F0E1FE0090AD
:108B6000102002F0DDFE009B13240190002B05D0A5
:108B700000280CD11324009802F0B2FD019B002BB9
:108B800002D0180002F0ACFD20000BB0F0BD1020A8
:108B900002F0C6FE0600102002F0C2FE13240500FB
:108BA000002E00D1AEE0002819D01022002102F0E2
:108BB00017FE32002900039802F0D2FE041E0ED1E7
:108BC00033787F2B51D830000099FFF7ABFF009B23
:108BD0001B787F2B53D801990098FFF7A3FF300033
:108BE00002F07EFD002D02D0280002F079FD002C5D
:108BF000C1D1102002F094FE0600102002F090FE79
:108C00000290002E7CD0002878D03A000F3223004A
:108C10000125121105D00F333B4015B25A42534182
:108C20001BB26A1E1201002B33D0049BD2B29818DB
:108C30000099029AFFF76CFF013D102200213000DD
:108C400002F0CEFDADB2049F2D017D19AF4242D09E
:108C5000002C33D0300002F043FD029B002B00D1EA
:108C600089E7180002F03CFD85E729003000FFF796
:108C700059FF28002549009AFFF74AFFA7E7290076
:108C80000098FFF74FFF28002049019AFFF740FFA7
:108C9000A5E70F210F4004998A18D9B28F4208D94D
:108CA000D15C06A819540133102BF6D1029A019910
:108CB000C0E7791A48424141C901F2E73900300062
:108CC00006AAFFF725FF3200039806A902F048FE26
:108CD00010370400BAE7002CBCD13000029906AA74
:108CE000FFF716FF320006A9039802F039FE0822AA
:108CF00004003100059802F0B3FEABE71324A9E7A6
:108D00001324AAE7002800D06EE733E770BE0011F5
:108D1000F0B58BB00F0016000225009000283FD060
:108D2000002A3DD00B1DDBB21800029302F0F8FDC3
:108D30001135041E34D0FDF747FD05003A000099B7
:108D4000201D02F06DFCEBB20393E3702B0CDBB241
:108D50002F0A00936370FFB22B0E2370A77001934C
:108D6000FDF72CFD1022010006A802F059FC21009D
:108D7000029A04AB06A8FFF7E9FE051E0DD1039B7E
:108D800008223370009B04A9B370019B7770F370C5
:108D9000301D02F045FCFDF71DFD200002F0A0FC97
:108DA00028000BB0F0BDF0B58FB00D00149E0390FD
:108DB00004920593002A03D1022420000FB0F0BDD5
:108DC000002EF9D00398FFF7E5FD1424071EF4D018
:108DD0007278337812021A43B3781B041343F27883
:108DE00012061A43036A0192934201D30133E3D17D
:108DF000002D03D03B7901249B07DED508220021FA
:108E000006A802F0EDFC059B13240433DBB2180026
:108E1000029302F085FD051ECFD0059A0499043017
:108E200002F0FEFB04223100280002F0F9FB3900B9
:108E3000102210310AA802F0F3FB2900029A06ABB7
:108E40000AA8FFF783FE041E0FD1082206A908A86E
:108E500002F0E6FB0822311D08A802F071FE01288D
:108E600007D101990398FDF7C9FC280002F038FCEE
:108E7000A3E70124F9E7000070B51C4C0500236846
:108E8000181E10D0002D14D11A78002A0CD1981C6D
:108E9000083202F0E5FD02F0FBFC0135002808D1A4
:108EA00023681D70012070BD0A331800082202F0EB
:108EB000D7FD2368002BF5D0122002F039FD061EE5
:108EC0000DD0C12321680370457002311022023099
:108ED00002F0C6FD23683100587802F0F1FB2068EB
:108EE00002F0FEFB00232360DCE7C0464C60FF1F5E
:108EF000F8B504002020FDF755FB0D4EA700BB5927
:108F00000500002B0DD000280BD0D878FF2809D100
:108F100008492A000C55F35907480333611802F039
:108F20009FFCF8BD290002F053FB0028F0D1F8E7C0
:108F30006860FF1F5060FF1F49A1001170B5064D0A
:108F400084006359002B05D0D87802F031FCFF2251
:108F50006359DA7070BDC0466860FF1F70B50600C7
:108F60008CB00C00150000213022684602F038FC5D
:108F700031001022684602F053FB1D20210003221D
:108F8000684402F04DFB6846FFF7D8FD2D21040030
:108F900003222800694402F043FB20000CB070BD9E
:108FA000F0B50700160097B001931CAB1D78302276
:108FB0001EAB00910AA800211C7802F011FC1022BF
:108FC00039000AA802F02CFB1022002102A802F0AE
:108FD00007FC0722310002A802F022FB072202ABA5
:108FE0009818631E9C41019902F01AFB02AB9C7316
:108FF0002B005A1E934102AAD3730021102206A807
:1090000002F0EEFB06221D9907A802F009FB1A20C8
:1090100002ABC01806221F9902F002FB1022009931
:109020000EA802F0FDFA102202AB0EA908781C78F7
:10903000013A6040D2B2087001330131002AF5D103
:109040000AA8FFF77BFD102212A904000EA802F067
:1090500007FD102206AB0EA908781D78013A68407A
:10906000D2B2087001330131002AF5D10AA8FFF706
:1090700065FD044310222098E4B212A902F0D0FA50
:10908000200017B0F0BD70B50E0014008CB00100C8
:10909000102268461D0002F0C3FA3100082204A81D
:1090A00002F0BEFA2100082206A802F0B9FA6846CA
:1090B000FFF744FD04001022280008A902F0B0FACE
:1090C00020000CB070BDF8B506000D000024371963
:1090D000AC4200D3F8BD02F033FC030A3B70631CC2
:1090E000DBB201379D4203D90234F054E4B2EEE71B
:1090F0001C00EDE773B506000C000225002819D00E
:10910000002917D0032101A8FFF7DDFF6B469A79EC
:109110003F231A40013313436A463000937101A97B
:109120002200FFF71BFF051E04D10322E01C01A94A
:1091300002F096FC280076BD03785807DA08C00FC5
:10914000D20080009B0710439B0F1843C0B27047AA
:1091500007230B40C908C9000B4303707047000088
:1091600070B50400FFF7EAFE134DA4006359002B0D
:1091700021D0186A002801D002F0B2FA2B59986E5B
:10918000002801D002F0ACFA2B59D86E002801D08B
:1091900002F0A6FA2B59186F002801D002F0A0FAAD
:1091A0002B59586F002801D002F09AFA285902F082
:1091B00097FA00232B5170BD6860FF1F0E4B800093
:1091C000C35870B50C00002B0FD09D68002D0CD03B
:1091D0002B78201D0B706B784B70A97CFFF7B8FFC4
:1091E0002B7E23726B69E36070BD1022002120008A
:1091F00002F0F6FAF8E7C0466860FF1F014B1860FE
:109200007047C0466460FF1F074A03008000825811
:1092100010B5002A06D0D088984203D1012901D187
:10922000FFF79EFF10BDC0466860FF1FF0B5264ED9
:1092300095B087000B93BB590500099112200A9243
:10924000002B31D0D888FFF7A5FB04001420002C98
:109250002AD0280010A9FFF7B1FFBB591E781D6A5C
:10926000002E23D00895FDF7EFFA07000020FDF748
:10927000F1FA0790A379E61D069310AD0CA90898A2
:1092800000F0E2FA0EA9280000F0D7FA0B9B0A9929
:109290000493069B09980293079B039601930097FA
:1092A0000EAB0CAAFFF77CFE15B0F0BDFDF7CCFAB3
:1092B00006903000FDF7CEFAE31DA779079310ABB7
:1092C00006000893DAE7C0466860FF1F30B50C4C13
:1092D00085002A59030085B00120002A0ED018000D
:1092E0006946FFF76BFF2B591A78D888054B002A7F
:1092F00000D1054B6A46072100F0D9FB05B030BD0F
:109300006860FF1F3B9800114998001130B5094C67
:109310008500295985B010226846253102F0A0FB4E
:109320002A591121044BD0886A4600F0C0FB05B0D1
:1093300030BDC0466860FF1FE598001130B5094C8C
:109340008500295985B010226846353102F088FB26
:109350002A591121044BD0886A4600F0A8FB05B0B9
:1093600030BDC0466860FF1F23990011F7B54D4F0F
:1093700086001020F4590D0002F0D2FAF359206251
:10938000186A132200286CD0033A29009C6802F066
:1093900067FBF3591A780192002A58D11E6A227D80
:1093A000317B944651400122019F114201D1674611
:1093B0001740217D914339432175377B4F40BC468F
:1093C00060460027800701D44F0817400121022082
:1093D0008F40227D82433A432275377B5740BC46FB
:1093E00060460027400701D497080F400420227DE3
:1093F000BF0082433A432275627D0027944660464F
:10940000727B42400A4201D167460F400121627DD2
:109410008A433A436275777B5740BC4660460027D3
:10942000800701D457080F400220627D7F008243ED
:1094300017436775767B00227E40760701D4BA0811
:109440000A400426617D9200B1430A4362756A783E
:10945000002A08D06278002A05D005220533DA7781
:1094600000221000FEBD04222979114205D1A17C01
:10947000114202D10533033AF1E7019A21782C78A1
:10948000002A02D10A002100140018220429E8D879
:10949000042CE6D805206043034A05331218525CB9
:1094A000DDE7C0466860FF1F80BE001110B50A00EE
:1094B0001121024B00F0FBFA10BDC0467F9900114C
:1094C0000B0030B587B001AD2B806B460400110056
:1094D000981D082202F0C4FA2A000B212000024B3A
:1094E00000F0E5FA07B030BDA799001110B50A00E9
:1094F0001121024B00F0DBFA10BDC046FB990011B0
:1095000013B50B0011006A4613706B460400062267
:10951000581C02F0A5FA6A4608212000014B00F011
:10952000C6FA13BD1B9A001110B50A001121024B97
:1095300000F0BDFA10BDC0466B9A00117FB5050062
:109540000B4BAA00D4580800002C0FD0666F237F65
:10955000E28821780396266F0296E66E0196A46E45
:109560000094FDF709FC2800FFF7FAFD7FBDC04617
:109570006860FF1F10B51721FFF7E0FF10BD000066
:1095800070B50A000D00064B0221040000F08FFAAE
:10959000060029782000FFF7D1FF300070BDC046DB
:1095A0004B99001170B586B000236A46137083682A
:1095B00004001D78681E0A2859D801A902F010FA83
:1095C000060633373B3F43474B4F5300180000F02C
:1095D00042F9062312284BD000281BD16088FFF7E0
:1095E000D9F90823002813D04279002A47D1264B05
:1095F0001A78072312070BD5244B1A680723002A71
:1096000006D01668002E03D0290001AAB047030037
:109610006A4613706B461B786088002B2AD1FFF7CF
:1096200067FC06B070BD180000F06CF9D4E71800B4
:1096300000F087F9D0E7180000F093F9CCE71800A4
:1096400000F0ADF9C8E7180000F0C3F9C4E718004E
:1096500000F0F6F9C0E7180000F0F6F9BCE71800D2
:1096600000F013FAB8E7180000F013FAB4E7072384
:109670006A46137069466088FFF782FFD1E70523C9
:10968000012AC5D1024BB8E7F55EFF1F6060FF1FDE
:109690006460FF1FF8B52C4F8600F35904000D00DD
:1096A000002B40D0DA8882423DD15A78062A33D145
:1096B0001A78002A2ED0012099681A6A097D014281
:1096C00006D0157B054203D007225A700120F8BD51
:1096D0000220014204D0157B054201D00922F4E7A3
:1096E0000420014204D0127B024201D00B22ECE79D
:1096F000164B1B68002BE9D05B68002BE6D02000DE
:109700009847BB5900215B78122BDFD12000FFF76F
:1097100015FFDBE70E4BECE7112A04D1002900D03E
:1097200032252900F2E7002D08D12000FFF732F999
:10973000002803D01023027913430371210028006D
:10974000FDF798FAC2E7C0466860FF1F6060FF1F20
:109750006460FF1F70B50E4E8500AB590400002BEE
:1097600013D01B78002B11D10A4B1B68002B04D09F
:109770005B68002B01D02000984773595B78122B4F
:1097800003D100212000FFF7D9FE70BD024BECE7AA
:109790006860FF1F6460FF1F6060FF1F094B80004F
:1097A000C3581020002B0CD01A6A002A09D09B68DD
:1097B000002B06D0127A1B7E101C9A4200D9181C6E
:1097C000C0B270476860FF1F70B503000D00140041
:1097D0000220002A30D000292ED013700B78081DEB
:1097E00053704B789370FFF7A7FCE07001200221C3
:1097F0002B7A23716B7B034063716A7B0A401343AE
:10980000042263716E7B1640334363716E7BF608EE
:10981000F600334363712B7B0340A371287B014027
:1098200000200B43A371297B0A401343A3712A7BB9
:10983000D208D2001343A37170BD10B50A00010015
:109840000120FFF7C1FF10BD10B50A000100022082
:10985000FFF7BAFF10BD70B506000C000220002E05
:1098600030D000292ED07378201D0B70B3784B7048
:10987000F178FFF76DFC01223579257271794B1073
:1098800008001340934010400343881010408000AC
:10989000C9080343C9000B436373B1794B10080037
:1098A0001340934010400343881002409200C908BF
:1098B0001343C9000B4321202373FCF773FE854239
:1098C00001D2122070BD2220257AFCF76BFE854262
:1098D000F7D823781820042BF4D86378012BF1D81B
:1098E0000020EFE7030010B50220002909D0002B6B
:1098F00007D00322481C0A7019000D3202F0B0F89C
:10990000002010BD03000222080010B5002B06D075
:10991000002904D00E32591C02F0A2F800221000D7
:1099200010BD030010B50220002909D0002B07D07C
:109930000422481C0A7019000C3202F091F8002031
:1099400010BD10B5FFF7DEFF10BD03000220002997
:1099500006D0002B04D0052200200A701B784B7023
:10996000704703000220002B08D0002906D05B7846
:1099700000200B70013B082B00D918307047030002
:1099800010B50220002909D0002B07D00622481C60
:109990000A7019000A3202F063F8002010BD10B5F9
:1099A000FFF7B0FF10BD02000B00022010B5002928
:1099B0000ED0002A0CD00721197011885970118817
:1099C000090A997011180822D81C02F049F80020E1
:1099D00010BD03000A00022010B5002B0CD0002996
:1099E0000AD099785878090201431180901CD91C3B
:1099F000082202F035F8002010BD030010B5022047
:109A0000002909D0002B07D00822481C0A70190031
:109A1000921802F025F8002010BD02000B00022071
:109A200010B500290BD0002A09D00921197011782E
:109A300018185970511C062202F012F8002010BDAF
:109A400010B5FFF75FFF10BD02000B00022010B53C
:109A5000002A09D0002907D0517819701118062260
:109A6000581C01F0FDFF002010BD030010B50220BE
:109A7000002909D0002B07D00A22481C0A701900BF
:109A8000063201F0EDFF002010BD10B5FFF73AFFE0
:109A900010BD02000B00022010B5002A06D00029DC
:109AA00004D018005178FFF753FB002010BDF0B52B
:109AB00085B017001E006A46062305000800918144
:109AC0009380FEF7C0FC1324011E02900CD03800D6
:109AD000B047041E05D1280001A9FEF76FFA041E45
:109AE00002D0029802F034F82800FFF701FA2000B3
:109AF00005B0F0BDF0B504008BB001911500002158
:109B0000102202A801F06CFE334EA700B8590028BD
:109B10003CD0C388A34239D10378002B36D1427898
:109B2000062A18D102000100553235310C3006AB3F
:109B3000FFF7A9FA002829D12000FFF72FFE020025
:109B400006A902A801F08CFF200002A901F048FD3F
:109B500001200BB0F0BD816E002917D00B8A112AAD
:109B600028D19D420ED101981231093A01F0E8FF47
:109B7000012807D1BB5920009D6EFFF70FFE290079
:109B80000200DEE732212000FFF7D8FC2000FEF7BC
:109B900001FF061E1BD0416A002918D00B8AAB4278
:109BA00015D108220198123101F0CAFF01280ED107
:109BB000716A0AE09D42E9D108220198123101F050
:109BC000BFFF0128E2D1BB59996E8A7EB9E7200018
:109BD00001F0C6FDBCE7C0466860FF1FF0B56B4DE5
:109BE00087007E5985B0337802900393002B00D014
:109BF00087E0B368346A01937078062817D1012290
:109C00001B7D134202D0217B114218D10222134244
:109C100002D0217B114251D10422134203D0237B75
:109C2000134200D08BE0019B5A7DEB5991E007383D
:109C30000428F8D801F0D4FE032E42678300B36EE7
:109C4000002B03D11C2001F06BFEB066EB599C6E1B
:109C5000002C1CD010220021200001F0C1FD029830
:109C6000FFF79CFD01002000FFF72DFA01F068FED0
:109C70002082200008211230FFF725FA0298FFF712
:109C80008DFDA076EB592100D888FFF70FFC082244
:109C9000EB591CE0B36E002B05D01A00198AF0882E
:109CA0001232FFF70DFC0222019B197DEB59114284
:109CB0003DD0207B10423AD0073208E0F488FCF710
:109CC000DBFD01002000FFF711FC0A22EB595A705E
:109CD000029B9C002A595378073B042B11D8D0884B
:109CE000FEF758FE00284ED0C3895A08D2182849DA
:109CF000029B0298CB542B5941180433254801F09C
:109D0000AFFD05B0F0BDFCF79FFD030001208342CD
:109D100001D100200393EB59DE88FCF79BFD0399EA
:109D200002003000FFF7ECFB019AEB59117D042291
:109D300011420CD0217B114209D00B22C7E7F688D3
:109D4000FCF73CFD01003000FFF7EEFB6BE7019AEA
:109D5000527D01210A4204D0607B084201D00C22CE
:109D6000B5E702210A4204D0607B084201D00E22EE
:109D7000ADE704210A4204D0627B0A4201D01022DE
:109D8000A5E71222A3E7FA225200B0E76860FF1F9E
:109D90006C60FF1F53A1001110B5064B1A78042305
:109DA000100018401A4200D00348FFF727FA00209D
:109DB00010BDC046F55EFF1FB43DFF1F70B5040027
:109DC000FFF7D4FA051E43D12000FFF77FFA234E98
:109DD000A400A0598268937CDB0708D50321036A9D
:109DE0001B790B40012B02D1017F0B430377431DED
:109DF000D97F8B1E022B0DD8022900D00121C088EB
:109E0000FCF790FF042133591A7F59700A431A77DF
:109E1000280070BD01290CD10223102243700021BB
:109E20000C3001F0DDFC305910213530FFF74BF9D3
:109E3000EEE70529ECD10223D118437010220C3033
:109E400001F00EFE04233259117F0B431377EAE72A
:109E500008251828DCD1053DDAE7C0466860FF1FF9
:109E6000F0B58BB0059143887E4F9E00F4591500E4
:109E70000493002C15D1012902D000200BB0F0BDB5
:109E8000101D57781678FFF757F9EB6832000293E8
:109E90002B7A0499019300903B002000FCF70CFF03
:109EA000EBE7E388049A934201D00820E6E72378A1
:109EB000012B00D1D4E0059B581E092800D9CFE022
:109EC00001F08EFD05CE0A29CC506C859AB229008E
:109ED0000498FFF773FFD1E72000290010224530D6
:109EE00001F0BEFDB9594B78042B02D1013B4B70F8
:109EF000C3E70B000A00253335320C310498FFF715
:109F000095F90498FFF702FA0522431E9841BB59C0
:109F1000C0005A70B2E7200029001022553001F02D
:109F20009FFD049B4F4C9D00295904980A0006ABE5
:109F300055320C31FFF77AF929591022453106A81C
:109F400001F0FEFD012808D10498FFF7F7F905900C
:109F5000002804D106222B595A7005988EE7082351
:109F60000593FAE763780C2B7AD1E36E002B03D1CB
:109F70001C2001F0D5FCE066BB59D86E00286FD0DC
:109F80001022290001F06CFDBB590498DC6EFFF72C
:109F900005FC0D22A076BB595A706EE7E06E0028D2
:109FA0005ED063780D2B5BD12B8808220382A91C1D
:109FB000123001F055FDBB599A68517D02221142C1
:109FC00026D0186A407B104222D00C32E4E7637836
:109FD0000E2B45D1236F002B03D1162001F0A0FCDE
:109FE0002067BB59186F002803D01022290001F008
:109FF00037FD0F22BB59CFE763780F2B30D1206F8D
:10A000000622691C103001F02BFDBB599A68517D66
:10A010000422114203D0196A497B1142D5D1002193
:10A020000498FFF78BFA28E7636F002B0DD0BB591C
:10A03000586F0028F3D01022290001F011FD0122F1
:10A04000BB5952425B6F1A61E9E7142001F068FCCA
:10A05000BB5960675B6F002BE9D126E72978DFE702
:10A0600007200BE76860FF1F10B5064C207001F059
:10A07000CFFB06212078FDF791FF0348FEF778FC1F
:10A0800010BDC0467B60FF1F0992001100200BB27B
:10A0900070B50D00834216DA264B187801F048FBA4
:10A0A000041E0DD00378922B0ED0A02B37D0224B5C
:10A0B0001878FF283AD0210001F002FB002835D1A2
:10A0C00080200002684070BD43780E2B0BD03E2BE1
:10A0D000EDD18378052B12D0082BE8D181798088C7
:10A0E000FFF7D8FA08E0154B82889A42DFD18368DF
:10A0F0001878591CFEF7C0FE002817D1D7E7104B7F
:10A100001B785B0712D50F4B1B68002B0ED09B688A
:10A11000002B0BD0C289811D80889847ECE7FFF7A0
:10A1200041FAA068002801D001F012FD200001F0E2
:10A130004FFCC5E77B60FF1FAD3DFF1F18200000EF
:10A14000F55EFF1F6460FF1F10B50078FFF712FA7D
:10A1500010BD10B50078FFF7FDFA10BD0C23434386
:10A16000084A10B59B185A68002A03D0012901D16A
:10A17000904710BD9B68002BFBD00029F9D1984770
:10A18000F7E7C0469860FF1F01238340094A10B5D6
:10A19000946B1C439463506B98435063D46B2000C2
:10A1A0009843012901D120001843D063116B0B4360
:10A1B000136310BD00800040F0B500240127154B4B
:10A1C00085B0DA6B144E03921A6C0192DA64019B2B
:10A1D000E3403B4217D0039DE5403D400295E5B288
:10A1E00002992800FFF7BAFF316A736A002908D084
:10A1F0003900002B01D0029979402800FFF7C4FFF5
:10A2000001E0002BF9D101340C36172CDFD105B059
:10A21000F0BDC046008000407C60FF1F064B01215E
:10A220005A68C2400A4204D01B68C3401800084064
:10A2300070471B6DF9E7C046008000400122064BC5
:10A240008240002903D0D9680A43DA607047D96890
:10A250009143D960FAE7C0460038004030B5032486
:10A2600044430F4BE25C1B199C785D7801232D1B46
:10A270000135AB40013BA340A140DB430C00122859
:10A2800007D80849920052181168194021431160FB
:10A2900030BD054A11680B4023431360F8E7C04600
:10A2A000C7BE001108F0004014F00040C21F70B596
:10A2B000D4B20623092C0BD80125084C954000295F
:10A2C00008D00021FFF7CAFF23682B432360002337
:10A2D000180070BD2368AB43F8E7C0460038004063
:10A2E000214BF0B51B185B78022B21D1032444438A
:10A2F0001E4A1F4EA35C1219947801221500854056
:10A30000B76B013CE4B23D43A240B563194C12283F
:10A3100015D89B0000290CD117495B1899680A438E
:10A320009A600123205C154A834011680B43136037
:10A33000F0BD11495B18996891439960F1E70E4BA4
:10A3400000290DD159690A435A61225C1328E8D0CB
:10A350000123203A93400A49086803430B60E7E76A
:10A36000596991435961F0E77C60FF1FC7BE001136
:10A37000008000400CBF001100F00040A0F0004041
:10A38000A4F00040F8B500241B4E1C4D1C4B1B5D77
:10A39000012B1FD1194A9269E2401A420BD00122C7
:10A3A000B25693402200143AD2B2022A09D8154973
:10A3B0004A6913434B61013402360C35172CE5D141
:10A3C000F8BD0022B2560F499200521891680B4313
:10A3D0009360F0E7022BEED1E7B23800FFF71EFFE3
:10A3E00001235840C1B23800FFF77AFF3800FFF769
:10A3F00015FF6877DFE7C04699BE00117C60FF1F3C
:10A400007D60FF1F00F00040012202388240054BB2
:10A41000002903D059690A435A6170475969914329
:10A420005961FAE700380040F8B50E0001210F002D
:10A430008740114A0400D368FD43BB43D360831EA9
:10A440008B4201D8FFF7E0FF00212000FFF72EFF2D
:10A450000A4A0B4B5168012E05D139431B19516033
:10A460005E700020F8BD2940516002221C19627004
:10A470009A6915409D61F4E7003800400080004073
:10A480007C60FF1F012210B58240074B002906D0D7
:10A4900019680A431A600121FFF7C6FF10BD196849
:10A4A00091431960F7E7C046008000400C2370B567
:10A4B000002543430A4A29009B181D70094B0400DC
:10A4C0001B185D70FFF7B0FF0123A3400649280069
:10A4D0000A681A430A6005490A689A430A6070BD0F
:10A4E0009860FF1F7C60FF1F348000403080004078
:10A4F00070B504000E00FF2813D003250540FFF7B8
:10A50000D5FF084AA3089B009B183F22ED00AA40F4
:10A51000AE40196820009143314319600121FFF7D3
:10A520008DFE70BD18380040F8B50C244443134B21
:10A530000500E4186368002B03D1A3681220002BE8
:10A540001AD0022201270E4B00215B195A702800F5
:10A550002770FFF769FF63681E1E08D0A3683E00DE
:10A56000002B04D02800FFF759FE4640F6B2280021
:10A570003100FFF709FE0020F8BDC0469860FF1FBC
:10A580007C60FF1FF7B5C420FF222B4B80001958B9
:10A59000002491433F3A0A431A508022274F520227
:10A5A000274E1A60274B1D5D002D21D0A31E012BC5
:10A5B00003D80121E0B2FFF727FF012D18D11F4B6F
:10A5C0009B69E3402B4213D0E3B218000193FFF7DD
:10A5D00025FE01000198FFF755FFE3B2143B022B63
:10A5E0001DD801217156184A8D405369AB43536100
:10A5F0003B7F002B0DD0E5B22800FFF795FF280028
:10A60000FFF70CFE7B7F0100834202D02800FFF79A
:10A61000A5FD01340C370236172CC3D1F7BD01213B
:10A6200000237156F3568D40074A9B009B189A6889
:10A63000AA439A60DCE7C04600E100E07C60FF1FAF
:10A6400099BE00117D60FF1F00F0004070B50E0044
:10A6500015000400FFF72AFF0C236343094A20007A
:10A660009B189D605E60FFF75FFFF021064B074A75
:10A670008900051E5A5002D02000FFF717FF28005E
:10A6800070BDC0469860FF1F0000FF1FB9A10011F8
:10A6900070B5134D07202C78002C1FD19822210073
:10A6A0005200280001F0C4F80123C420FF222B70BF
:10A6B0000C4B80001C635C630B4B1C605C600B4BA1
:10A6C000195891433F3A0A431A50802252021A60A5
:10A6D0000D20074A074901F07BF8200070BDC046F5
:10A6E0007C60FF1F00800040A0F0004000E100E01F
:10A6F00085A5001185A3001170B51D0002240C2949
:10A7000010D8094ACA40D2070CD5FBF757FF041EE0
:10A7100008D1059A04992800FBF76CFFFCF7DAFDD5
:10A72000FFF73AFB200070BD1210000030B50D7825
:10A7300002232C009C43184201D02B431C00082507
:10A740002300AB43284201D02B00234320241D00CB
:10A75000A543204201D01C4325002A230D70184236
:10A7600004D011781E3B0B43137030BD0028FCD180
:10A770000C2113788B43F7E7F8B51D0006AB1B8857
:10A78000140007AA0E000B201778002B27D10A7897
:10A79000022A49D14A68507811780002244A0843B5
:10A7A0008018042840D801F01BF903121D1B230058
:10A7B000F06801F035F9021CC0B2B84200D93A1C69
:10A7C000D2B22000F1682A8001F04AF906E00222A4
:10A7D000F3681B882A8023701B0A63700020F8BD71
:10A7E0000622EEE701232B80F3681B782370F5E740
:10A7F000F368002B16D008222A801A8822701A8843
:10A80000120A62705A88A2705A88120AE2709A88F4
:10A8100022719A88120A6271DA88A271DB881B0A97
:10A82000E371DBE72B80D9E701202B80D7E7C04617
:10A8300000D6FFFFF7B516000A781D0008AB1F8889
:10A840000C000123022A18D14A68507811780002BE
:10A850002B4A0843801803280FD801F0C1F80225BD
:10A860004439E06801F0DCF8C0B20723B84204D3F1
:10A870007B190193152B02DD0D231800FEBDE06846
:10A880002A003100C01901F0EBF86B4600209B88CC
:10A89000E268D0541B4B1B68834203D01B68834281
:10A8A00000D098470023E8E70B23002FE5D1022DC5
:10A8B000E2D1737832781B021343E2681380114BA4
:10A8C0001B68002BEED01B68002BEBD00120E8E7C3
:10A8D0000B23002FD1D1062DCED12A003100E06804
:10A8E00001F0BEF8DEE70B23002FC6D1012DC3D146
:10A8F00032787533012AC0D8E3681A70D2E7C046AF
:10A9000000D6FFFF8862FF1F70B50C0015000728F6
:10A9100037D801F065F8041436361B36242E18207B
:10A9200015290BD8184E16220021300000F058FFD0
:10A9300022002900300001F093F8002070BD18209B
:10A940000229FBD11288114B1A80F6E7182008293A
:10A95000F4D10A000E48290001F0AAF8EDE718200A
:10A960000129EBD10B4B10780B49DA69FFF7DEFEBA
:10A97000E3E718200129E1D1064B10780749DA6B8B
:10A98000F4E70220DAE7C0467062FF1F563EFF1F61
:10A990004C3EFF1FDC3DFF1F043EFF1F243EFF1FF8
:10A9A000030010B50020DB0704D50721024A034845
:10A9B00000F08CF810BDC04624BF0011DC3DFF1F25
:10A9C000054A03001068002803D082889A4201D10A
:10A9D000806870470068F6E78064FF1F0A880300FC
:10A9E00008009A4204D08A8804309A4200D000209D
:10A9F00070470000F8B5F22200230D4F0D4E796824
:10AA0000050042433370994200D07B600A4C00211C
:10AA1000200000F0E5FE00231A007C60AB4202D16A
:10AA200000203370F8BD01332280DBB2F234F5E749
:10AA30007865FF1F7665FF1F8464FF1F73B56B4643
:10AA400001900600684615001980FCF775FF041E8A
:10AA500011D1002D0FD07689002E11D00C2000F0DE
:10AA60005FFF00280ED0084A046013688680856066
:10AA7000002B02D11060200076BD1A001B68F7E79A
:10AA80000224F8E71324F6E78064FF1F0121002267
:10AA90000A4B10B549420A4C198099809A719A70F4
:10AAA000084B2070012019805A60FFF7A3FF20781F
:10AAB000FCF7A0FF0448FDF75BFF10BD9062FF1F8D
:10AAC0008065FF1F7865FF1F79AB0011022310B569
:10AAD000002802D0FFF7B2FF0300180010BD0000ED
:10AAE000030010B50020DB0704D50421024A034807
:10AAF000FFF7A4FF10BDC04638BF00115C3EFF1F2A
:10AB0000F0B50E2687B003930CAB1F8802ABF61886
:10AB10000500080031000292FDF790F804000120C2
:10AB2000002C0FD03088FFF74BFF03000E20002BC6
:10AB300008D05E68002E05D021002800039B029AF1
:10AB40000097B04707B0F0BD0A4B10B5984207D147
:10AB50000122002352420A808B708A808B7110BDC3
:10AB6000FFF73CFF0028FAD001235B42038000235B
:10AB70008370F4E7FFFF0000F8B5050001290AD152
:10AB8000134E00243388F227AB4219D02800114914
:10AB9000FFF7DAFF06E0022904D10139FDF766FF6D
:10ABA0000028EDD0F8BD3B0063437268D018D35A3B
:10ABB000002B09D03A00002100F012FE0134E4B26B
:10ABC000054B1B78A342EED801235B423380DDE7BF
:10ABD0007865FF1F9062FF1F7665FF1F10B5FFF7B6
:10ABE000FDFE03000020834200D0987810BD0000D5
:10ABF000F0B589B01C000EAB80CB03901E8810AB63
:10AC00001B78049202930B7A0D00DB0616D42B7886
:10AC10000593022B24D00498FFF7D2FE002812D00F
:10AC200003689C46002B0ED0029B22000193290052
:10AC30003B00644603980096A04705E00498FFF7A0
:10AC4000BFFE002802D10E2009B0F0BD8368002BA2
:10AC5000F9D00A222900039898470028D7D0F3E7B3
:10AC60006B6858781A786B4B000210439842D2D820
:10AC7000043B984210D2684B984242D015D8674B9B
:10AC8000C0180128C7D80B20002EDDD1EB681A7838
:10AC900059683A80200028E0614BC018032800D989
:10ACA00079E000F09DFE846A789E5E4B9842B2D1B6
:10ACB0000B20002EC8D101233B80EB6831001B78AC
:10ACC00023706889013080B2FCF7B8FF3A88031E10
:10ACD0000ED0017802328A183A8042896270428925
:10ACE000120AA27059680278E01C00F0B9FE06E072
:10ACF00004323A8031000422601C00F071FD002013
:10AD0000A2E70B20002E9FD1EB6807A91E88042321
:10AD10003B80330A300026706370FCF78FFF051EFE
:10AD200028D004AB9A890E2304A95B183E49C66853
:10AD3000FCF7F8FF00280BD12B783C486A6805998E
:10AD4000FBF7AEFB002803D1012304AA5B42D381A9
:10AD50003278022A06D17168201D00F081FE3B88FE
:10AD600002333B800E2304AA9B181B88A3701B0A86
:10AD7000E370C4E704ABDE81F4E70B20002E00D0C3
:10AD800062E7E9680398FFF729FF02233B80207000
:10AD9000000A6070B3E70B20002E00D054E70222B7
:10ADA000EB681B883A8023701B0A6370A7E7E8688A
:10ADB00000F036FEC2B203000720B24200D243E7E1
:10ADC0000DD00299DBB27118994202DB921BD3B20B
:10ADD0000293029BE9681A003B8089195AE7002315
:10ADE000F6E70B20002E00D02EE70722EB683A8012
:10ADF0001A7822705A7862705A88A2705A88120A99
:10AE0000E2701A792271DA886271DB881B0AA371F9
:10AE100075E7C046042900000228000000D8FFFFA3
:10AE2000FFD6FFFF03280000FFFF000068BE0011EF
:10AE3000F0B58DB06B460020089120229B5E8342C6
:10AE40003DDAA64B187800F073FC071E32D0037869
:10AE5000B02B2CD10079023816281FD800F048FEFC
:10AE600017001E001E001E0031001E0096001E006E
:10AE70001D011E0052011E0073011E00CD011E00A7
:10AE800050021E001E001E008E021E00E302944BA4
:10AE900094491B8878880B80FBF742F83800FCF750
:10AEA000C3FF914B1B68002B01D038009847380036
:10AEB00000F08EFD8020089B0002434018000DB07A
:10AEC000F0BDEE220021874800F08AFC0BAA3B7BF4
:10AED0007989388900923A000D32FCF7C7FD0400E9
:10AEE000804B1B78002C3FD146E0804B788805933F
:10AEF0007F4B4100CB5A0BAE073BDBB2328802934B
:10AF0000002301937B4B210006930093059BFFF7E1
:10AF10006FFE744D002810D1069B3A8A1B889A4216
:10AF20000BD138000599123000F00AFE002804D039
:10AF30002B7862899B00EB185A80162306A81B18F1
:10AF4000328820007989FCF7EDFE2B7804009A0006
:10AF5000AA1851880029C3D00133DBB22B70002816
:10AF600007D006A9C98A9180634A12889A42BCD840
:10AF700002E0012149429180002B04D05949788890
:10AF8000FBF702F88AE73E890A2479E000253E892A
:10AF9000574B06937B88069A5B009B5A033B9D4266
:10AFA00002DB002DF0D05BE0162206A812183B7BD6
:10AFB000798900923A0030000D32FCF757FD059078
:10AFC000002858D04689017A7888FCF719FD041EBC
:10AFD00044D1464B78880793069B4100C95A454B9C
:10AFE0000439C9B206AAD28A069302910194009349
:10AFF0000599079BFFF7FCFD041E2FD1069B3949DD
:10B000001A88931C002D26D14B807988384B490033
:10B01000CB5A5119033B8B4220DD059B31485B899C
:10B0200041190B71A91C0135C9B2EDB20591451941
:10B030001B0A2B71059B2D490433181800F010FDD5
:10B040002C4B059A1B88D318DDB22C4B9E4205D0A1
:10B050000136B6B29CE749889942D6D0002D0CD073
:10B06000204C2800618800F083FB20702100788844
:10B07000FAF79AFF12E7059CF0E7002C00D183E76E
:10B080007B78142B00D109E716493B794E800B7071
:10B090000C717888FAF73AFF00E7162406ABE4183B
:10B0A00021003889FCF7CAFD011E00D1B7E178887C
:10B0B00022880F4C45002C5B0A4D013CE4B20294FF
:10B0C00000240F4B01940095FFF792FD041E00D061
:10B0D00014E129007888FAF777FFDFE68065FF1F23
:10B0E0004C3DFF1F9862FF1F8C62FF1F8C63FF1F88
:10B0F000C85EFF1F7C64FF1F4A3DFF1FFFFF00006B
:10B100009A62FF1F162406ABE41821003889FCF769
:10B1100095FD011E00D182E178882288AE4C450061
:10B120002C5BAE4D013CE4B202947C89AC4B0194A3
:10B130000095FFF75DFD041E00D0DFE02900788850
:10B14000FAF74CFFAAE60025A44B1D803B00F6331E
:10B150001B78A24A78880792AB4208D99E4B128886
:10B160000693069943005B5A013B9A4203DB079919
:10B17000FAF73EFF92E616246B00FB18059306AB28
:10B18000E418059B21001889FCF758FD011E03D126
:10B19000059B01241E8973E77888924B2288069CC0
:10B1A000099343001B5B904E013BDBB202930023EB
:10B1B00000960193099BFFF71BFD041E02D0059B1F
:10B1C0001E895DE77B88069A5B009B5A079A108868
:10B1D00032881218934202DC1B1A013B33807F4CE9
:10B1E000023032880999001900F03AFC238832882D
:10B1F00001359B182380EDB2A8E70BAA3B7B798928
:10B20000388900923A000D32FCF730FC0025059099
:10B21000059B002B04D10A24002D00D16EE060E0D4
:10B22000059B7888197AFCF7EBFB0100041E63D1BB
:10B23000694C6C4B788806940993069B4400E45A49
:10B24000694B063CE4B20BAE32880793029401913D
:10B2500000930599099BFFF7CBFC041E4CD1079B7B
:10B260005E491B881A1D002D30D14A80059B5B4C1E
:10B270005A8963191A716B1C9BB2E318120A1A716E
:10B28000162306A832881B1879890598FCF74AFD11
:10B29000FF21AA1C2E1D03350B00059092B2B6B2F9
:10B2A000ADB2002803D006ABDB8AD9B21B0AA218C4
:10B2B000651911712B714C4D301D2A884949201890
:10B2C00000F0CEFB2B88F618B5B2A1E74988914271
:10B2D00007D17A8806995200525AEB18053A9A42D9
:10B2E000C4DC3E4C2800618800F0EAFB207021009D
:10B2F0007888FAF787FED1E5002DF2D13E89BFE6C6
:10B30000162606ABF61831003889FCF797FC3D008D
:10B310000400FA3500282DD0037A9B060CD40022B5
:10B320007B893989788800923A000C32FFF7E8FB74
:10B33000041E10D03E8915E03088FFF741FB00283D
:10B340001AD08368002B17D02100122278889847E2
:10B35000041EE4D0EEE72B78002B02D17888FAF7B0
:10B3600061FE00262B78002B00D097E5002C00D141
:10B3700094E585E60124DDE70E24DBE7162506AB20
:10B38000ED1829003889FCF759FC041E47D0037AD0
:10B390009B0611D4154A7B881188994203D0144822
:10B3A000814207D11380134BF2261D780023D9B2B6
:10B3B000A94221D30924A1E72888FFF701FB00282F
:10B3C0002FD08368002B2CD0210012227888984738
:10B3D000041EDFD092E7C046C85EFF1F9862FF1FC1
:10B3E0009A62FF1F8C63FF1F7C64FF1F7865FF1F3D
:10B3F000FFFF00007665FF1F310059435468013399
:10B400006018615A0029D2D13C0008342100F22290
:10B4100000F026FB21007888FAF70CFE3EE50124B7
:10B420006CE70E246AE71D4B1A887B889A4231D05C
:10B430007888FAF709FE31E5F2230598516843430D
:10B44000CD18C95A00291FD03B7A012B0BD16C882B
:10B45000AB887888AA1D0094FFF752FB041E02D027
:10B4600000233B722E88F2220021280000F0B8F958
:10B4700000232B80059B0133DBB20593084B059914
:10B480001B78064A8B42D7D801235B421380002CDD
:10B49000CED0F5E5002634000596EFE77865FF1F6E
:10B4A0007665FF1F70B504000E001500FFF796FAD1
:10B4B000031E08D131000548FFF790FA0300112060
:10B4C000002B02D01C8000209D7070BDFFFF00008B
:10B4D000F8B50B4F06003B780D001400FF2B0ED083
:10B4E0000A2000F025FA011E09D0B12303800023B1
:10B4F00046800371C5800481387800F0E1F8F8BD1A
:10B500009D3EFF1FF7B50F0008A90600088809A98E
:10B510000B240988002821D10234022B1ED1557832
:10B5200013782D021D432B008B4301937334002BA2
:10B5300014D1FB68300019000093FFF74FFB019C0A
:10B5400085420BD02A0030000099FFF7ABFF041EA4
:10B5500004D12A0030007989FFF7BAFF2000FEBD30
:10B56000F0B50E7885B003900AA805880120022E58
:10B570000DD14C682778647824023C43054FBC42C7
:10B5800005D10398DBB201960095FFF7BBFF05B02C
:10B59000F0BDC04602290000034B10B51B68002B0C
:10B5A00000D09847FEE7C0468465FF1F07B501A895
:10B5B000FFF7F2FF044A05480021121A00F038F99B
:10B5C000F8F718F9FEE7C0468865FF1FA03EFF1F89
:10B5D00001B40248844601BC604700BF51470100E6
:10B5E00001B40248844601BC604700BF311B000023
:10B5F00001B40248844601BC604700BF3936FF1FD2
:10B6000001B40248844601BC604700BF3935FF1FC2
:10B6100001B40248844601BC604700BFC51D00005C
:10B6200001B40248844601BC604700BF4551010097
:10B6300001B40248844601BC604700BF1D4B0100B5
:10B6400001B40248844601BC604700BFA533FF1F18
:10B6500001B40248844601BC604700BF456B01004D
:10B6600001B40248844601BC604700BF350E0000AB
:10B6700001B40248844601BC604700BFE528FF1FB3
:10B6800001B40248844601BC604700BF090E0000B7
:10B6900001B40248844601BC604700BF791800002D
:10B6A00001B40248844601BC604700BF691F000026
:10B6B00001B40248844601BC604700BF55490100FF
:10B6C00001B40248844601BC604700BF594F0100E5
:10B6D00001B40248844601BC604700BFC521000098
:10B6E00001B40248844601BC604700BF014C010020
:10B6F00001B40248844601BC604700BF6571010087
:10B7000001B40248844601BC604700BF6DBC000024
:10B7100001B40248844601BC604700BF8D1200009E
:10B7200001B40248844601BC604700BF212DFF1FC1
:10B7300001B40248844601BC604700BFF54E0100D9
:10B7400001B40248844601BC604700BFF92AFF1FCC
:10B7500001B40248844601BC604700BFC94A0100E9
:10B7600001B40248844601BC604700BF091B0000C9
:10B7700001B40248844601BC604700BF350E00009A
:10B7800001B40248844601BC604700BF6D33FF1F0F
:10B7900001B40248844601BC604700BF5D17000049
:10B7A00001B40248844601BC604700BFA54F0100B8
:10B7B00001B40248844601BC604700BF1147010044
:10B7C00001B40248844601BC604700BF59520100E1
:10B7D00001B40248844601BC604700BF812BFF1FB3
:10B7E00001B40248844601BC604700BF154D01000A
:10B7F00001B40248844601BC604700BFC9A90000EB
:10B8000001B40248844601BC604700BF6532FF1F97
:10B8100001B40248844601BC604700BFC92600004D
:10B8200001B40248844601BC604700BFE533FF1FF6
:10B8300001B40248844601BC604700BFB70E000057
:10B8400001B40248844601BC604700BF392BFF1F8A
:10B8500001B40248844601BC604700BF055E000099
:10B8600001B40248844601BC604700BFA9460100FC
:10B8700001B40248844601BC604700BF75A90000BE
:10B8800001B40248844601BC604700BF2526000081
:10B8900001B40248844601BC604700BFD91B0000C8
:10B8A00001B40248844601BC604700BF2146010044
:10B8B00001B40248844601BC604700BF792EFF1FD7
:10B8C00001B40248844601BC604700BFB130FF1F8D
:10B8D00001B40248844601BC604700BFC56D010049
:10B8E00001B40248844601BC604700BFADAE000011
:10B8F00001B40248844601BC604700BF3D18000007
:10B9000001B40248844601BC604700BFB14E00004C
:10B9100001B40248844601BC604700BFE117000043
:10B9200001B40248844601BC604700BF3D4B0100A2
:10B9300001B40248844601BC604700BF1D4D0100B0
:10B9400001B40248844601BC604700BF2951010090
:10B9500001B40248844601BC604700BFBD30FF1FF0
:10B9600001B40248844601BC604700BFE5480000BE
:10B9700001B40248844601BC604700BF9134FF1FF8
:10B9800001B40248844601BC604700BFB54C0100C9
:10B9900001B40248844601BC604700BFE9280000AA
:10B9A00001B40248844601BC604700BFED4A010073
:10B9B00001B40248844601BC604700BFF94C010055
:10B9C00001B40248844601BC604700BF5125000015
:10B9D00001B40248844601BC604700BF434D0100EA
:10B9E00001B40248844601BC604700BF4D36FF1FCA
:10B9F00001B40248844601BC604700BFF30E00005A
:10BA000001B40248844601BC604700BF492DFF1FB6
:10BA100001B40248844601BC604700BF0D520100DA
:10BA200001B40248844601BC604700BFDD520100FA
:10BA300001B40248844601BC604700BF5118FF1F93
:10BA400001B40248844601BC604700BF851F000066
:10BA500001B40248844601BC604700BF4D1F00008E
:10BA600001B40248844601BC604700BFE94C0100B4
:10BA700001B40248844601BC604700BF8552010002
:10BA800001B40248844601BC604700BF4550000035
:10BA900001B40248844601BC604700BF7D18FF1F07
:10BAA00001B40248844601BC604700BF291C000065
:10BAB00001B40248844601BC604700BF810E00000B
:10BAC00001B40248844601BC604700BF090E000073
:10BAD00001B40248844601BC604700BFE12AFF1F51
:10BAE00001B40248844601BC604700BF9DA9000024
:10BAF00001B40248844601BC604700BF6136FF1FA5
:10BB000001B40248844601BC604700BFB352010043
:10BB100001B40248844601BC604700BF0124000014
:10BB200001B40248844601BC604700BFEDA5000097
:10BB300001B40248844601BC604700BF156B010098
:10BB400001B40248844601BC604700BFCD4C0100EF
:10BB500001B40248844601BC604700BFD9490100D6
:10BB600001B40248844601BC604700BF21240000A4
:10BB700001B40248844601BC604700BF355500004F
:10BB800001B40248844601BC604700BFDD66010085
:10BB900001B40248844601BC604700BF8B520100DB
:10BBA00001B40248844601BC604700BF0D35FF1F49
:10BBB00001B40248844601BC604700BFB131FF1F99
:10BBC00001B40248844601BC604700BFE130FF1F5A
:10BBD00001B40248844601BC604700BF5522000002
:10BBE00001B40248844601BC604700BF2534FF1FF2
:10BBF00001B40248844601BC604700BF5933FF1FAF
:10BC000001B40248844601BC604700BF017F0000C8
:10BC100001B40248844601BC604700BF056A0000C9
:10BC200000030103020203030402050006020700E9
:10BC3000080009020A030B030C000D000E030F039A
:10BC4000100311031300140015031603BD3B00116C
:10BC5000F13B0011000000000200000062BC001176
:10BC6000192A0F180A000000F1590000FD240000F5
:10BC700041460100798000118DA00011E17400118E
:10BC80007D7E0011F152001131AE0011594F0011AB
:10BC9000B13D0011E13E0011000000001616000049
:10BCA00002000000ACBC0011F4FFF3FFD2FC000066
:10BCB000214000110000000000000000547579616F
:10BCC0000042312E340030303138006769746875B5
:10BCD000622E636F6D2F707676780054483035434E
:10BCE0000000000002000000F8BC0011292A282AE8
:10BCF000272A262A252A242A0A180000E2040000FE
:10BD00007102000078EC0000744000001027000071
:10BD100060F0000006640000204E000000000000FB
:10BD2000050000001F501D00023CB4000001180077
:10BD300014000000A10200003031323334353637B0
:10BD4000383941424344454600000000F556001191
:10BD500049570011000000000200000064BD0011FE
:10BD60006F2A6E2A1A18EAD8BC80F0FC6000000026
:10BD70000000000000005F066B2F363D7D077F3F0F
:10BD8000777C596E7971AF066D4FC6CBEB0EEFCF56
:10BD9000EEC3A966E9E8FA60D6F46CBCBEE0FEFC2E
:10BDA000EE3E9A769E8E000001A00000000000008A
:10BDB0006410B71DC8206E3BAC30D9269041DC76AC
:10BDC000F4516B6B5861B24D3C7105502083B8ED56
:10BDD00044930FF0E8A3D6D68CB361CBB0C2649B7A
:10BDE000D4D2D38678E20AA01CF2BDBDFB349B5F9F
:10BDF000800000800010000000000000E3600011DF
:10BE00006D77001107610011757B00118B610011C6
:10BE10004B7B001101620011217B00115362001164
:10BE2000E97C0011BB620011E97C0011ED62001198
:10BE3000A37C001101620011D97A0011796200110E
:10BE4000817C001100000000000000005F63001111
:10BE5000817C0011C163001185770011052A042A35
:10BE6000012A002A022903280128002801180018A5
:10BE7000000000000000000000000000000000873B
:10BE80000101020102010102010203030401030195
:10BE9000010101010303020103000D000E00100067
:10BEA000110013001401070108010A010B011C0114
:10BEB0001D02040205020702080219021A021C02EE
:10BEC0001D03010302031700020100050400080717
:10BED000000B0A001716001D1C01020101050401D8
:10BEE0000E0D011110011413011716011A19020287
:10BEF00001020B0A020E0D02111002141302171692
:10BF0000030504030807030B0A030E0D00010203D7
:10BF100007090A0B0E0F101112141718191A1B1FFC
:10BF20002021220079A7001135A80011000000008F
:10BF3000020000006EBE00110000000061B500119B
:0CBF400000000000020000006CBE0011B8
:020000041FFFDC
:1000000000000000193D001168BC001164BC001123
:10001000AC5BFF1F000000000000000000000000BB
:1000200000000000000000000000000000000000D0
:1000300000000000000000000000000000000000C0
:1000400000000000000000000000000000000000B0
:1000500000000000000000000000000000000000A0
:100060000000000000000000000000000000000090
:100070000000000000000000000000000000000080
:100080000000000000000000000000000000000070
:100090000000000000000000000000000000000060
:1000A0000000000000000000000000000000000050
:1000B0000000000000000000000000000000000040
:1000C0000000000000000000000000000000000030
:1000D0000000000000000000000000000000000020
:1000E0000000000000000000000000000000000010
:1000F0000000000000000000000000000000000000
:1001000000000000000000000000000000000000EF
:1001100000000000000000000000000000000000DF
:1001200000000000000000000000000000000000CF
:1001300000000000000000000000000000000000BF
:1001400000000000000000000000000000000000AF
:10015000000000000000000000000000000000009F
:10016000000000000000000000000000000000008F
:10017000000000000000000000000000000000007F
:10018000000000000000000000000000000000006F
:100190006D2DFF1FCD2BFF1FC16601000000000069
:1001A000000000000000000000000000000000004F
:1001B000000000000000000000000000000000003F
:1001C000000000000000000000000000000000002F
:1001D000000000000000000000000000000000001F
:1001E000000000000000000000000000000000000F
:1001F00000000000000000000000000000000000FF
:1002000000000000000000000000000000000000EE
:1002100000000000000000000000000000000000DE
:1002200000000000000000000000000000000000CE
:1002300000000000000000000000000000000000BE
:1002400000000000000000000000000000000000AE
:10025000000000000000000000000000000000009E
:10026000000000000000000000000000000000008E
:10027000000000000000000000000000000000007E
:10028000000000000000000000000000000000006E
:10029000000000000000000000000000000000005E
:1002A000000000000000000000000000000000004E
:1002B000000000000000000000000000000000003E
:1002C000000000000000000000000000000000002E
:1002D000000000000000000000000000000000001E
:1002E000000000000000000000000000000000000E
:1002F00000000000000000000000000000000000FE
:1003000000000000000000000000000000000000ED
:1003100000000000000000000000000000000000DD
:1003200000000000000000000000000000000000CD
:1003300000000000000000000000000000000000BD
:1003400000000000000000000000000000000000AD
:10035000000000000000000000000000000000009D
:10036000000000000000000000000000000000008D
:10037000ADB500110000000000000000000000000A
:10038000000000000000000000000000000000006D
:10039000000000000000000000000000000000005D
:1003A000000000000000000000000000591AFF1FBC
:1003B000000000000000000000000000000000003D
:1003C000000000000000000000000000000000002D
:1003D000000000000000000000000000000000001D
:1003E000000000000000000000000000000000000D
:1003F00000000000000000000000000000000000FD
:081838009069FF1F4118FF1F1A
:10184000024981F3088801F0F7FF00009069FF1F4B
:1018500010B502F011F8072804D0122808D0022889
:1018600008D010BD044A0420136B01331363F8E75A
:101870000220F6E71420F4E7705FFF1FF8B50700B9
:101880000C0026002500503630785135002804D150
:101890000300287058342370F8BD2978CA00481E08
:1018A0008141A3183800A25C5B68C9B2FFF7D0FF82
:1018B00000280DD12B78DA00A218013350602B706C
:1018C0003378044A013B3370136A01331362D8E75B
:1018D0000123DFE7705FFF1F5C234343074910B517
:1018E000C9180B0058331B78012B05D1FFF7C6FF31
:1018F000034A936A0133936210BDC046A45FFF1F81
:10190000705FFF1F10B502F07FF8064A0121130037
:1019100010CB4942D967044B136001F06DFF2000E2
:1019200010BDC04600E100E01000100010B504003A
:1019300002F06AF8024B1C6001F05EFF10BDC04669
:1019400000E100E0431E5A425341A022F0B5D2010B
:101950005B421340154D164A40019B182A18127E0F
:101960008BB00191002A1BD01A000832D46F0022DC
:10197000E6B206AFE4B294420EDC2818C369002B2D
:1019800008D0019902AA117106AA049202AA16733C
:1019900003A898470BB0F0BD1978B9540132EAE7B3
:1019A0001A7D1A7806AB01261A70E6E73062FF1F2F
:1019B00000400040F0B5254B04004001C25C85B0FA
:1019C000002A2BD01A18117E002927D0917E0029D9
:1019D00024D01179022921D11689D788D168F51B25
:1019E000ADB22A1C102D00D9102292B2BE4217D1DE
:1019F0001818012303710023C269C38003819A422E
:101A000006D06846032103730171029301A8904731
:101A10000820002C00D0192001F08EF805B0F0BD90
:101A2000013C65426C41A0256442ED012C40084D0B
:101A30001B186419074D0633013A92B2AA42EDD041
:101A40001888461C1E80085C2070F5E73062FF1F76
:101A500000400040FFFF00000F220E4B10B59868B9
:101A6000104002380A280BD801F0F0FD0D0A0B0ACD
:101A70000A110A0A0A0A060002210020FFF762FF83
:101A800010BD0121F9E70020FFF794FFF8E7DB6FB5
:101A9000F6E7C046004000400F220E4B10B5986894
:101AA000104002380A280BD801F0D0FD0E0A0B0AAC
:101AB0000A120A0A0A0A060002210120FFF742FF61
:101AC00010BD01210800F9E70120FFF773FFF7E7D8
:101AD000DB6FF5E700900040564B70B51B68012B9B
:101AE00003D1554A936D0133936501F005FF534BC4
:101AF000534A1860534B544C1A600123534A1360E5
:101B0000534A13602378002B06D0062251495248CD
:101B100001F0A2FE00232370504A514B10681B783D
:101B2000C1B2002B0ED14F4CC0B223785BB2002B58
:101B30004FDB237824785BB264B21B0424021B19A8
:101B40001B1813600B1C50294ED95023464A474995
:101B50001078DBB2FF2202284BD10868444C454D77
:101B6000267890432A78964254D9227824782E7881
:101B7000023B5D10A31B6B435201D31A10335B1160
:101B80001843086001F028FF031F012B45D83A4B8A
:101B90001B78002B06D0394B1B78002B02D000207D
:101BA00001F02AFFA122364B92009978354B4A4327
:101BB0001B689B18832292009B181B78033B012B08
:101BC00003D8AF20400001F08FFD01222E4BDA82B6
:101BD00070BD237824785BB264B2FF33FF341B04FA
:101BE00024021B190138ABE7CAB2022AAED2022383
:101BF000ACE70868254C264D267890432A78964213
:101C000008D9227824782D78023B5B10641B63434B
:101C10005201B2E72378DBB2B2E70228D5D11D4BDF
:101C20001B78013B022B03D91B4B1B78022BCCD119
:101C30006C20C8E79809FF1FFC0FFF1FA85EFF1F5D
:101C4000FF3F000014100340AC5EFF1F0C10034068
:101C500000100340D50BFF1F7211FF1FB40003409B
:101C60008C09FF1F680AFF1F490AFF1F94000340E9
:101C7000460AFF1F470AFF1FF908FF1F2209FF1F1F
:101C8000300DFF1F3409FF1FBC0BFF1F440AFF1F4D
:101C9000450AFF1F1C09FF1F2309FF1F10B501F094
:101CA0008BFE0022014B1A8010BDC046A65EFF1FAE
:101CB00070B5244D2B68002B28D001F04DFD2B680A
:101CC000D8402B680400002B27D001F0A5FE2B681C
:101CD000D8401D4B1D4A9978A1239B004B431268A5
:101CE000D118D25C91239B00002A20D0CA5801321F
:101CF000CA50174B17491B680868834214D3D23B5C
:101D0000181A012A1AD0144B186070BD01F024FD76
:101D1000124B196801F0C0FCD3E701F07DFE0F4BB8
:101D2000196801F0B9FCD4E70D495B18E8E7CA501F
:101D30000C4B1B68DB68E418201AE4E7F530FF3031
:101D4000E1E7C0461C08FF1F300DFF1F3409FF1FCD
:101D50009C09FF1FA85EFF1FA009FF1F1808FF1F97
:101D60002DFF3F00B05EFF1F70B504000D00282955
:101D700016D10300A433C2881B889B1A0B4A9BB25E
:101D800093420DD906006A3605223100653001F014
:101D900003FE002804D13100200001F025FE70BDB3
:101DA0002900200001F040FDF9E7C046FE7F000059
:101DB000F8B50500012001F0BFFD134CA36AA26A2B
:101DC0009342FBD1114E336001F076FC10490300C1
:101DD00008601048426894460F4A17680022BC45C4
:101DE00001D24268BA1A0D4802603268AD18A422C6
:101DF000E562606A520302436262094A1278002A6D
:101E000001D00F3B0B60F8BD00F00040340AFF1F0B
:101E1000E408FF1F28100040180AFF1F1C0AFF1FBC
:101E20001C09FF1F70B580241025E405A3682B430F
:101E3000A36001F049FCA368AB43A36070BD000040
:101E4000F7B5160080221C001023D205019191687D
:101E500005000B43936000225A4BD7301A6001F003
:101E60008BFC9D232A002F009B00EB58CA320121D6
:101E70000092FC37002B01D00021009A386801F055
:101E80000BFD2900009BCB311A784F4BD3351A60DC
:101E90004B780A781B0213438A7812041A43CB78D2
:101EA0001B061343494A1BBA13604B790A791B027C
:101EB00013438A7912041A43CB7931001B0613436A
:101EC000434A1BBA13606B782A781B021343AA7823
:101ED00012041A43EB781B0613433E4A1BBA1360E5
:101EE000019A330213433C4A13603C4B22001B1BF4
:101EF0009C4603293DDCB3089A0013005142B21AF4
:101F0000032A46D1354AE018511A827840781204E3
:101F100000020243E05C043302430A600022FF2B0C
:101F20004BDDF0222E4B12011A600F222D4B1A604E
:101F30002D4A1368002BFCD00023224A2749136046
:101F4000091B321D0B191B68043A180A23706070B4
:101F5000180C1B0EA070E3700434002AF2DC8022FF
:101F600010213B68D20501333B6093688B4393603B
:101F7000F7BD6346D578981893782D061B042B433C
:101F8000157804392B43557804322D022B43036016
:101F9000AFE7022A0AD1114AE05C511AE2185278DE
:101FA000120202430A6004339BB2B7E7012AB5D19B
:101FB0000A4A521AE15C1160F5E7084959180A60AB
:101FC0000433ACE7000004403C0004403800044007
:101FD00034000440300004400C0004400001044080
:101FE000040004401000044014000440F7B515003C
:101FF00080221C001023D2050091916807000B433A
:1020000093600023654AD730136001F0B5FB9D2330
:102010003E009B00F9583B00CA363200FC330029D1
:1020200000D07FE0586801F037FC390032785C4B13
:10203000CB311A604B780A781B0213438A78AC467E
:1020400012041A43CB78281D1B061343554A1BBAAA
:1020500013604B790A791B0213438A7912041A43DD
:10206000CB791B061343504A1BBA13604B7A0A7A8A
:102070001B0213438A7A12041A43CB7A21001B06EF
:1020800013434A4A1BBA1360009A2B021343484A6F
:1020900013602200474B1B1B0093009BCE785B18FC
:1020A00001938B7836061B0433430E780438334390
:1020B0004E78043136023343019E33600328ECDC52
:1020C0000321A808431C9B002940800003292BD131
:1020D0003849E5185E18A9786D78E35C09042D028B
:1020E000294319433160030008330021FF2B2DDD04
:1020F000314B324919600F21314B196001232749B7
:102100000B60304B19680029FCD006211B680B407E
:10211000042B20D080220020D20593680A318B4303
:102120009360FEBD01217DE7022908D121495D1898
:10213000E1184978E35C090219432960D3E70129D2
:10214000D3D11C495918E35C0B60CCE71948181827
:1021500001600433CAE7002310490B606346002B7B
:102160000CDC3B00FC335A68102101325A6080229B
:10217000D205936801208B439360D2E7009B9B18A4
:102180001B68190A13705170190C1B0ED3700423AD
:102190005B4291709C440432E0E7C046000004407A
:1021A0003C00044038000440340004403000044047
:1021B0000C0004400001044004000440080F00002B
:1021C000100004401400044010B5002901D001F0B3
:1021D000D3FB10BDF7B5604B01919978A1239B000B
:1021E0004B435E4A060014681022E418D6235B00B5
:1021F000E0583623FF33E35C00279343222B41D181
:10220000574B0F3A1A600760012501F0DDFB019B77
:102210001880E8235B00E35C002B01D0B34258DD5B
:102220000023504FFB70AD33FF33E3581A68002A88
:1022300003D09B88DB439B071DD03823FF33E35C2F
:10224000002B18D09B235B00E35C002B13D1D13310
:10225000FF33E35CB3420EDAA4235B00E15AE018DB
:10226000090A023101F0A0FB23000122FE33013EE6
:1022700001351A87FA70E8235B00E35C002B2AD053
:10228000A8B2FEBD03683D00002BBED0818804309B
:10229000090A023101F088FBD6235B00E3581F6076
:1022A000B2E72300B133BA00FF3398580137818871
:1022B0000430090A023101F077FBE8235B00E35C9C
:1022C000BB42EEDCE822F61AED1800235200A354BC
:1022D000A6E70027F1E7200001F036FA00281FD01A
:1022E000002E1DDD7319882647190193B6002000C2
:1022F00001F002FA5A3080002018406801358188C8
:102300000430090A023101F04FFB200001F0ACFA61
:10231000A3590133A351BD4202D0019B9D42E6D196
:10232000114BE35C002BABD095239B00E35C002BAF
:10233000A6D00E4BE15A0029A2D00D4AA35C9942C7
:1023400002D90133A3549BE700231A212000A35490
:1023500001F0B2FA94E7C046300DFF1F3409FF1FA9
:1023600000140340E010FF1F5A0200007202000038
:102370005E0200000D4970B54A6E0D4CD2038B69A8
:10238000D20BA24206D80B4D0224AA4204D901F076
:10239000EBF970BD02246442E21815007E2425404A
:1023A0002242F4D0A3432B438B61F0E700F00040BE
:1023B0000A200000FC1C00000B001B3B70B5040051
:1023C0003020E02B0DD81300E025493BFF3B9BB2AA
:1023D000ED00AB4205D8034B200019825A8201F070
:1023E000D3F970BD8410FF1FD722044B92009B5875
:1023F00010B5002B00D0984710BDC0460000FF1F4D
:1024000010B501F0ADF8FFF7EFFF2749274BCA6D74
:10241000274C1A4084235B001343CB65254B1B6874
:10242000186A01F089FA244B244A1A60244B254A81
:102430001A60A022244B52001A60244B187801F035
:1024400023FA2000224901F01FFB0023A36002337E
:10245000A360204B2049236003232048A36001F0A0
:1024600013FB10221E4BFF201A60802252031A60B9
:10247000802292031A60802212041A6001F0BCFAD2
:10248000012001F011FAFA20400001F02DFA582045
:1024900001F02AF9134801F017FA012001F044F97C
:1024A000072001F019FA10BD00F0004000FEFEFF09
:1024B00014100040B05EFF1F000003400180063D85
:1024C000BC00034034080000A40003404A0AFF1F78
:1024D00071020000C3090000FFFF3F002810004008
:1024E00000E100E030750000674E336888331B68F8
:1024F00083F3088801F0C0F8644A65491368002036
:102500000B401360634B644A1B68934200D1A6E002
:1025100001F01AFA0221614A13688B431360FFF736
:102520006FFF5F4B5F4C1878C0B201F01DFA0023BB
:10253000A3600233A3605C4B0120236001F0FCF92F
:102540000323A36001F0E0F9040001F0D5F90500D0
:1025500001F0DAF9554B186001F06EFA544B196826
:10256000621A531EA14200D213008022D20393426A
:1025700001D39B029B0A3268D16AC90700D471E07B
:102580004C491C0C09689BB24C4359432402090A6C
:10259000641803264849FC3293680A6847489B1A26
:1025A000474A0768126847499B18474A9A183340B8
:1025B0009208DB190A600360042B03D9013233400F
:1025C0000A6003600E684149A619300001F064F802
:1025D0003F4F3E493B68C3183B603000019301F018
:1025E000E3F83C4E3068081838493060884205D915
:1025F000019B01333B6001F0D7F8316001F0DCF85A
:10260000354B1B78002B0DD001F076F9334B621B54
:10261000196812188A4232D24919091B091A30481E
:1026200001F032FA2F4E337A002B0ED001F064F90C
:10263000621BF1681218914224D94919091B091A21
:10264000294801F021FA00233372284B83F30888CC
:1026500001F062F8002001F077F901F02DFA01F0A5
:1026600073F95CE7DC0199000234641A5900641ABA
:1026700009214B438033CB40A408E41889E7FA21B1
:102680008900CCE71A49DBE7B05EFF1F1CF0004071
:10269000FFFFC1FF0C0AFF1FB641210310000040DD
:1026A000490AFF1F14100040C3090000100AFF1F51
:1026B000340AFF1F380AFF1F200AFF1F280AFF1FC6
:1026C0001C0AFF1F240AFF1FC4090000710200003A
:1026D0006008FF1F2C0AFF1F1C09FF1FE408FF1FD3
:1026E00000100040740BFF1F3C1000400000002051
:1026F000DC050000A022054B92009B5810B5002B72
:1027000001D0984710BD01F017F8FBE70000FF1F4C
:10271000A122054B92009B5810B5002B01D0984781
:1027200010BD01F009F8FBE70000FF1FA222054BD6
:1027300092009B5810B5002B01D0984710BD00F0B7
:10274000FBFFFBE70000FF1FA322054B92009B58F5
:1027500010B5002B01D0984710BD00F0EDFFFBE74E
:102760000000FF1FA422054B92009B5810B5002BC0
:1027700001D0984710BD00F0DFFFFBE70000FF1F0E
:1027800070B501F0B9F84F4B186001F06DF9040015
:10279000C30702D401F040F870BD00224A4B1A6012
:1027A0004A4B18780138042829D800F04FFF03203D
:1027B000181C2400200001F037F90128ECD0444C0B
:1027C0002378042B6ED100F06FFF0028E4D001F0D5
:1027D00063F9582000F088FF02232370DCE7200013
:1027E00000F0DAFFE9E7200001F036F9E5E7200024
:1027F00001F00AF8E1E7200000F06EFFDDE701F0EC
:10280000EBF80500012808D1324B1B78053B012B62
:1028100003D82000FFF76EFFD1E72D4B1B78022B6A
:1028200001D0052B20D1022D28D12B4B9B7BAB4314
:102830001CD12000FFF76CFF264B18780128BED171
:102840006405BCD4244925224B7B034205D1233A9D
:1028500013405A42534126331A000B7D9342AED99E
:10286000322000F0C1FFAAE7022D07D1194B1B78D7
:10287000052B11D12000FFF759FFDDE7012D0BD10A
:10288000012B03D12000FFF75FFF98E7062B03D150
:102890002000FFF767FF92E7200000F04DFF022DB8
:1028A0008DD1C9E7032B04D10C4B987C00F08CFF31
:1028B00072E7072B00D06FE7094B987B00F0C4FF4D
:1028C0006AE7C0469C09FF1F9809FF1F9009FF1F78
:1028D0002309FF1F1C09FF1FA60BFF1FBC0BFF1FB7
:1028E000D40BFF1F10B500F099FE10BDF7B50B0C0F
:1028F000FF270122009300233C001E001D00944688
:10290000019089B262469A4010000840184136187A
:10291000B6B2FF2F02D1012E00D19FB20098024023
:102920001A41AD18ADB2FF2C02D1012D00D19CB2DD
:102930000133102BE6D10320012E07D1012D04D144
:10294000019B2401E4191C700138FEBD102EFCD13E
:102950000238102DF9D00230F7E700008023F7B5D8
:102960009C46264B264F01932649274A274D284C43
:10297000284B02281AD1604638600868264E30403D
:10298000802636033043086001990978002909D16F
:102990001660224A2A60224A2260E0221968914386
:1029A000A03A1BE08021C9021160F2E766463E6052
:1029B0000F68194E3E408027FF023E430E6001998A
:1029C000097800290DD1176001280ED1154A2A6017
:1029D000154A2260E02219689143C03A0A431A60FE
:1029E000F7BD802189021160EEE7E0210F4A024322
:1029F0002A600F4A22601A688A43F0E74B0AFF1FD9
:102A0000E0000340D8000340900003400000034072
:102A10005000034040000340FFFFE3FF0280063DFB
:102A2000804508220180063D8066082200800698C5
:102A300080550822F8B51E4B80261A680020140025
:102A40003440324232D11A681A4F32431A6001229E
:102A50003B68063093433B6000F06EFF0122164D49
:102A60002B681E432E603B680A2613433B60802779
:102A7000BF00124B1B683B4211D1013EF6B2FF2E44
:102A800009D17E220E4B1C682B68E40B1440934343
:102A900023432B6005E0082000F04EFFE9E7002EFD
:102AA000EFD180222B68600893432B60F8BDC046AD
:102AB000C4F000405CF0004018F0004068F00040B6
:102AC00060F0004010B500F01FFE01215820034ABD
:102AD00000F0DAFDFFF7AEFF10BDC046600AFF1F31
:102AE00010B578220021034800F076FE00F0C4FF04
:102AF000002010BDB861FF1F70B5040000F084FF16
:102B000000230C200B4A010059438D18515C002909
:102B10000DD0A14208D1012300246B7000F034FFD6
:102B200000F06AFE200070BD01330A2BEBD11224A5
:102B3000F6E7C046B861FF1F70B5040000F064FFFF
:102B4000002319001D000D4A1078002806D0A0426D
:102B50000CD1557001310C320A29F5D1002B0AD164
:102B600000F08AFF00F048FE002070BD5078461E3D
:102B7000B0411B18EEE700F007FFF3E7B861FF1F55
:102B8000F7B504000C20002384460E4D01926746E1
:102B90005F43E85D7E19A04212D000280BD10A4B9A
:102BA0009C4662461B7808331370019B70707C55FD
:102BB0007160B360FEBD01330A2BE8D10320F9E751
:102BC0000720F7E7B861FF1FB461FF1F8020F8B549
:102BD000484BC0051B68C1248360474BFF251A681A
:102BE000012313434361454BA4001A68444B402121
:102BF0001A60444B1A68444B1A60444B1A59AA4352
:102C00001A51C52292009E58AE43314380269950F6
:102C10009F583F49F6010F403E439E509E588027E3
:102C20003602360A3043985080201A5900020A4072
:102C300002431A5104341A59364E3F04324080265A
:102C40003A431A511A5936061202120A32431A51DD
:102C500008341A5980260A4002431A51C3229200AE
:102C60009F58B446AF4337439F509F58294E0F405B
:102C700007439F509F5837408026360437438026AD
:102C80009F509F5836063F023F0A37439F50C0224D
:102C90001F59AF433A431A511A591202120A1643E6
:102CA000C6221E5192009C58AC4365462C439C5052
:102CB0009C5800250C4020439850C72080001A588B
:102CC000154C1140C02212020A431A50134B1B78B4
:102CD000DB08AB4201DC0020F8BD2378002B06D0D6
:102CE000A368002B00D0984701350C34EEE7122082
:102CF000F2E7C046D83DFF1FD43DFF1FB0F00040B3
:102D0000B061FF1FB4F00040AC61FF1F00E100E0C4
:102D1000FF00FFFFFFFF00FFB861FF1FB461FF1F4F
:102D2000030010B51F2809D80722002013400724EC
:102D300004490A78A24313430B7010BD00230620F8
:102D4000F5E7C046B461FF1F054B06491B780A68CA
:102D500005485B0702401B0B134300200B607047C4
:102D6000B461FF1F1CF00040FFFFC1FF70B50C25D0
:102D7000FFF7EAFF0A4B1C780A4BE4086543ED189D
:102D8000002C01D1200070BD2B78002B06D06B6881
:102D9000002B00D09847013C0C3DF1E71220F2E7F0
:102DA000B461FF1FAC61FF1F1FB5002102220B00A1
:102DB00001910091052000F077FE02230B490A687B
:102DC0001A42FCD120230393039B5A1E0392002B2B
:102DD000FAD1074A1368002BFCDA0B246C4420005C
:102DE000012100F0A1FD207804B010BD90C8004082
:102DF00000C8004013B504000A4B0193019B002B4F
:102E000001D1112016BDFFF7CFFF2300034004427C
:102E100005D0052000F090FD019B013BEDE7180077
:102E2000F0E7C046FFFFFF0707B500F0EDFD802289
:102E30000821D205936A0191002B01D107399162D3
:102E400002210C4A11600199481E01900029FAD113
:102E500003311160053101910199481E019000294B
:102E6000FAD11160002B02D18022D205936200F0CA
:102E7000C3FC07BD00C00040F0B52D4C89B02378DD
:102E8000002B4FD1FEF73EFD02232A4F03903A68F4
:102E90001A42FCD120230693069B5A1E0692002B51
:102EA000FAD1254E3368002BFCDA0120FFF7A2FF90
:102EB000011E02D0112009B0F0BD030003220190D1
:102EC000009005AD9F2000F0EFFD0321280000F0E9
:102ED0002BFD02233A681A42FCD120230793079B5B
:102EE0005A1E0792002BFAD13368002BFCDA01201E
:102EF000FFF780FF0028DDD10398FEF717FDAA78C1
:102F00006B7811041B020B4329780B436360130099
:102F1000113B0A49052B07D801239340A3600B609E
:102F2000012323700020C6E780231B03F6E7C04679
:102F3000C03DFF1F90C8004000C800409808FF1F18
:102F40001E4B30B55A6818781D4B85B0D3185942BE
:102F50004B4101210093002300F076FD194B1A4AE2
:102F600002259A6300221A6510325A658022C42114
:102F70009D65164B1648D202DA6789004258154BF8
:102F800080241A4080231B041343435064234120B0
:102F90000393E40500F006FA402000F003FA6562AE
:102FA000039D6B1E0393002DFAD103236362FFF789
:102FB0003BFFA562FFF760FF05B030BDCC3DFF1FB2
:102FC00095FFFEF700C80040050001FF04E100E0A6
:102FD00000E100E0FFFF00FFF0B585B00700FEF75D
:102FE00091FC022305002D4C22681A42FCD12023BB
:102FF0000093009B5A1E0092002BFAD1284E336892
:10300000002BFCDA0120FFF7F5FE002803D0112485
:10301000200005B0F0BD234B2360022322681A4232
:10302000FCD120230193019B5A1E0192002BFAD15F
:103030003368002BFCDA0120FFF7DCFE0028E6D124
:10304000194B1F60022322681A42FCD120230293ED
:10305000029B5A1E0292002BFAD13368002BFCDA35
:103060000120FFF7C7FE0028D1D1104B23600223B7
:1030700022681A42FCD120230393039B5A1E039219
:10308000002BFAD13368002BFCDA0120FFF7B2FEE7
:10309000041EBCD12800FEF749FCB9E790C80040E7
:1030A00000C8004001000006A8C8004001800001DF
:1030B00010B50020FFF790FF10BD000010B5064BC3
:1030C00018705960FFF73CFF00211320034AFFF7F7
:1030D00057FD002010BDC046CC3DFF1F412FFF1FF4
:1030E000F0B5040085B003920291FEF70BFC882234
:1030F00063035B0B52051A438023DB059D6A802323
:10310000274F0092BA68002601901B039A420CD9FF
:10311000F82326001B041E401C4206D08022214BAF
:1031200052025E6219680A431A60002D0BD100F04A
:103130006BFC02221C4B1A608023DB055A62013AA9
:103140009A6200F059FB0023039A934220D1002D8C
:103150000AD100F059FC144B03221D608023DB05CB
:103160005A629D6200F048FB8023BA681B039A42B2
:1031700008D9002E06D000220A4B0C495A621A6860
:103180000A401A600198FEF7D1FB002005B0F0BD9F
:10319000009A0299D2181278CA540133D4E7C04673
:1031A000C03DFF1F00C8004000C00040FFFFFEFF01
:1031B000F0B587B0029103920400FEF7A3FB0190E3
:1031C00000F022FC802302250122234EDB0535601E
:1031D0005D629A6200F010FB204F3B682B42FCD1ED
:1031E00020230493049B5A1E0492002BFAD11C4DF9
:1031F0002B68002BFCDA0120FFF7FCFD002802D031
:10320000112007B0F0BD2000039A029900F0A4FB42
:10321000022304003A681A42FCD120230593059B3F
:103220005A1E0592002BFAD12B68002BFCDA0120E4
:10323000FFF7E0FD051EE3D100F0E6FB802303224B
:10324000DB0535605A629D6200F0D6FA0198FEF700
:103250006DFBE0B2D5E7C04600C0004090C800401A
:1032600000C80040F0B5802489B00600FEF74AFB94
:10327000E405A36A02250393029000F0C5FB012335
:10328000304F3D606562A36200F0B6FA2E4C2368B1
:103290002B42FCD120230593059B5A1E0592002B3F
:1032A000FAD12A4D2B68002BFCDA0120FFF7A2FD92
:1032B000002803D01124200009B0F0BD244B236066
:1032C000022322681A42FCD120230693069B5A1E31
:1032D0000692002BFAD12B68002BFCDA0120FFF7B5
:1032E00089FD021EE6D11B4B03211E6003000190E5
:1032F0000090202000F0D8FB022322681A42FCD163
:1033000020230793079B5A1E0792002BFAD12B68A4
:10331000002BFCDA0320FFF76DFD041ECAD100F07C
:1033200073FB80230322DB053C605A629C6200F041
:1033300063FA039B002B01D1FFF776FD0298FEF79D
:10334000F5FAB8E700C0004090C8004000C800404F
:103350000100000694C8004007B500020191042254
:10336000000A01A9FFF724FF0EBD000073B5050098
:1033700005240B4AA3005B429B1819686B46DE1DAF
:103380003000FFF7B3FA022804D133782B55013C03
:10339000EFD276BD052CFCD00128FAD10230F8E737
:1033A000140900111F2807D8012380228340D20569
:1033B00091680B43936070473F2808D8012380220F
:1033C00020388340D20551690B435361F3E75F28EE
:1033D000F1D80123802240388340D205116A0B4383
:1033E0001362E8E71F2807D8012280218240C9051F
:1033F0008B6893438B6070473F2808D80122802157
:1034000020388240C9054B6993434B61F3E75F283D
:10341000F1D80122802140388240C9050B6A9343CC
:103420000B62E8E71F2810D880230200DB05153A5D
:103430001968012A06D820229143196019680A43A5
:103440001A60704701228240F6E73F2811D8802396
:103450000200DB05353AD968032A06D810229143C9
:10346000D960D9680A43DA60EBE70122203882404C
:10347000F5E75F28E5D842238022181A413B8340B4
:10348000D205516A99435162516A0B435362D8E79E
:1034900010B50400012813D1A022184992050B6829
:1034A0005B015B0913430B60154B164A1968114009
:1034B000154A0A431A60402219680A431A6010BD6F
:1034C0000028FCD101000A2000F0FEFA21000B20A8
:1034D00000F0FAFAC0220A4B920019680A43402110
:1034E0001A601A688A431A60B022044912060B68EF
:1034F0005B015B0913430B60E1E7C04614F0004039
:103500001CF000407F00FEFF80FD010072B6074AFC
:103510001368013313600422054B1A600023054A27
:1035200013608022D2055360FEE7C0467808FF1F73
:10353000C0F00040C4F0004005490B68002B05D1E5
:10354000044A0A6004490A60044A13607047C0468E
:10355000140AFF1F841E0000380AFF1FC4F0004039
:103560000023034A1360034A1360034A1360704741
:1035700054F0004040F1004044F10040002310B5F9
:10358000184C8AB0009301932378012B27D0694609
:10359000012000F0C1F9002817D1009B12490293C5
:1035A000019B06AA0393114B02A81B680493104BBE
:1035B0001B68059300F088F810220E4906A800F059
:1035C000EBF9002804D1FF23237000200AB010BDBE
:1035D0000123094A074902A8237000F075F8012069
:1035E000F4E7C046B45EFF1F10290011082900113E
:1035F0000C29001120290011B85EFF1F13B501240A
:103600006946012000F088F9034B00940193FFF70D
:10361000B5FF200016BDC046BB0B000010B5FFF77C
:103620009FFFFFF7EBFF002802D0024B984710BD29
:10363000FEE7C046E1A2000002B471464908490015
:10364000095649008E4402BC7047C04602B4714618
:1036500049084900095C49008E4402BC7047C046D5
:1036600003B47146490840004900095A49008E4494
:1036700003BC70470000000001B40248844601BC4E
:10368000604700BFC9A9000001B40248844601BCDC
:10369000604700BF0167010001B40248844601BCD5
:1036A000604700BF090E000001B40248844601BC17
:1036B000604700BF01D7000001B40248844601BC46
:1036C000604700BFBD5C010001B40248844601BCF4
:1036D000604700BFDD3F000001B40248844601BCE2
:1036E000604700BFF935010001B40248844601BCBF
:1036F000604700BF7912010001B40248844601BC52
:10370000604700BFD9B0000001B40248844601BC44
:10371000604700BFED68010001B40248844601BC67
:10372000604700BF7997000001B40248844601BC9D
:10373000604700BFE512010001B40248844601BCA5
:10374000604700BFE917010001B40248844601BC8C
:10375000604700BF71B0000001B40248844601BC5C
:10376000604700BFE90B010001B40248844601BC78
:10377000604700BFD1AE000001B40248844601BCDE
:10378000604700BF8944000001B40248844601BC80
:10379000604700BF116E000001B40248844601BCBE
:1037A000604700BF0934010001B40248844601BCEF
:1037B000604700BF090E000001B40248844601BC06
:1037C000604700BFD544010001B40248844601BCF3
:1037D000604700BF4DF9000001B40248844601BCB7
:1037E000604700BFB70E000001B40248844601BC28
:1037F000604700BF6137010001B40248844601BC44
:10380000604700BF9DA9000001B40248844601BC86
:10381000604700BFF535010001B40248844601BC91
:10382000604700BFDD0A010001B40248844601BCC4
:10383000604700BF51B8000001B40248844601BC93
:10384000604700BFB5B5001101B40248844601BC11
:10385000604700BFC1F7000001B40248844601BCC4
:10386000604700BFE94C010001B40248844601BC36
:10387000604700BF5976010001B40248844601BC8C
:10388000604700BFE927000001B40248844601BC3C
:10389000604700BFEDA5000001B40248844601BCAA
:1038A000604700BF2144000001B40248844601BCC7
:1038B000604700BF6911010001B40248844601BCA1
:1038C000604700BF53B9000001B40248844601BC00
:1038D000604700BF8D11010001B40248844601BC5D
:1038E000604700BFF90D010001B40248844601BCE5
:1038F000604700BF8512010001B40248844601BC44
:10390000604700BFC95C010001B40248844601BCA5
:10391000604700BF156B010001B40248844601BC3A
:10392000604700BFE1AC000001B40248844601BC1E
:10393000604700BF3D71010001B40248844601BCEC
:10394000604700BF0189000001B40248844601BC01
:10395000604700BF016C010001B40248844601BC0D
:10396000604700BF9573010001B40248844601BC62
:10397000604700BF8914010001B40248844601BCBD
:10398000604700BFE9D4000001B40248844601BC8E
:10399000604700BF21A9000001B40248844601BC71
:1039A000604700BFCD4C010001B40248844601BC11
:1039B000604700BFC115010001B40248844601BC44
:1039C000604700BF8D82000001B40248844601BCFC
:1039D000604700BFCD0C010001B40248844601BC21
:1039E000604700BFDD0C010001B40248844601BC01
:1039F000604700BF85C1000001B40248844601BC95
:103A0000604700BFED6B010001B40248844601BC71
:103A1000604700BF75A9000001B40248844601BC9C
:103A2000604700BF6D0B010001B40248844601BC31
:103A3000604700BF0134010001B40248844601BC64
:103A4000604700BFC166010001B40248844601BC62
:103A5000604700BFC56D010001B40248844601BC47
:103A6000604700BF0534010001B40248844601BC30
:103A7000604700BFBD0B010001B40248844601BC91
:103A8000604700BFADAE000001B40248844601BCEF
:103A9000604700BF2D6C010001B40248844601BCA0
:103AA000604700BF6DF6000001B40248844601BCC7
:103AB000604700BF496D010001B40248844601BC63
:103AC000604700BF8552010001B40248844601BC32
:083AD000604700BF5DA2001178
:103AD800020000006ABE00110100000058BC00117D
:103AE8000200000066BE001101000000183BFF1F25
:103AF8000200000060BC0011010000002C5CFF1FE8
:103B08000200000064BE001103000000A05BFF1F5C
:103B180012000000020000006ABE0011010000004F
:103B2800A0BC00110200000066BE001101000000E8
:103B38009DBC001102000000AABC00110300000097
:103B4800DB5BFF1F0200000064BE001103000000E1
:103B5800F05BFF1F0200000066BE001101000000BC
:103B68009CBC001102000000A8BC0011030000006A
:103B7800B15BFF1F0200000064BE001103000000DB
:103B8800D25BFF1F020000006ABE001101000000A6
:103B9800E4BC00110200000066BE00110100000034
:103BA800613CFF1F02000000F6BC0011010000008C
:103BB800DBBC00110200000066BE0011010000001D
:103BC800603CFF1F02000000F4BC0011010000006F
:103BD800F85BFF1F0200000066BE00110100000034
:103BE8005F3CFF1F02000000F2BC00110100000052
:103BF800CBBC00110200000066BE001101000000ED
:103C08005E3CFF1F02000000F0BC00110100000034
:103C1800C6BC00110200000066BE001101000000D1
:103C28005D3CFF1F02000000EEBC00110100000017
:103C3800C1BC00110200000066BE001101000000B6
:103C48005C3CFF1F02000000ECBC001101000000FA
:103C5800BCBC0011020202020202000000000000C7
:103C6800141300009D4B0011634B001138BD001167
:103C780090011D0018001800FFFF0701020304054A
:103C8800060201060000000000000000000000001D
:103C9800000000000000000000000000000000001C
:103CA80003000000020000006ABE001101000000CD
:103CB80058BD00110200000066BE0011010000009E
:103CC8001C3DFF1F0200000062BD00110100000042
:103CD800265CFF1F0200000064BE00110300000004
:103CE800905EFF1F0200000066BE00110100000088
:103CF8001C3DFF1F0200000060BD00110100000014
:103D0800285CFF1F0200000064BE001103000000D1
:103D1800885EFF1F12006C6C0000000000000000AD
:103D28000000000008070000000100000000011169
:103D3800FFFF000050485936000000000000000056
:103D48000B000500F0000000B4000028002800283F
:103D58003075A000A000A000A00000080008E00145
:103D6800F0001000100010001000100010005000AB
:103D78005000500010001000D007000000000000A4
:103D88000F0001000500307507001000010081FFD9
:103D980000000000FF000000457400114D72001182
:103DA800DD6F0011FFFF0100FF000000619E0011A0
:103DB800DD9B0011F59A00110000000000000000D2
:103DC80000000800040000003B0001085902E0015F
:103DD80088212800020000006ABE001101000000CE
:103DE80030BF00110200000066BE00110100000093
:103DF800593EFF1F0200000062BE001101000000D2
:103E08007062FF1F0200000066BE00110100000082
:103E1800583EFF1F0200000060BE001101000000B4
:103E2800563EFF1F0200000066BE001101000000A0
:103E3800543EFF1F020000005EBE0011010000009A
:103E48004C3EFF1F180018001D00900102000003DF
:103E580002020000020000006ABE0011010000001A
:103E680044BF00110200000066BE001101000000FE
:103E78009C3EFF1F020000005CBE00110000000015
:103E8800000000000200000064BE001103000000F2
:063E98009062FF1F20FFF5
:040000051FFF184180
:00000001FF
